:020000040800F2
:1000000068080020ED010008916800089368000866
:10001000976800089B6800089F68000800000000BF
:10002000000000000000000000000000A3680008BD
:10003000A568000800000000A76800080502000885
:10004000070200080702000807020008070200086C
:10005000070200080702000807020008070200085C
:10006000070200080702000807020008070200084C
:10007000070200080702000807020008070200083C
:10008000070200080702000807020008070200082C
:10009000070200080702000807020008070200081C
:1000A000070200080702000807020008070200080C
:1000B0004126000807020008292600080702000858
:1000C00007020008070200080702000807020008EC
:1000D00007020008F11F0008412C00080702000871
:1000E000636600080702000807020008070200080C
:1000F00007020008070200080702000807020008BC
:1001000007020008070200080702000807020008AB
:10011000070200080702000871270008070200080C
:10012000070200080702000807020008070200088B
:1001300000F002F800F04AF80AA090E8000C8244AF
:100140008344AAF10107DA4501D100F03FF8AFF28C
:10015000090EBAE80F0013F0010F18BFFB1A43F0A5
:1001600001031847809E0000A09E0000103A24BFA3
:1001700078C878C1FAD8520724BF30C830C144BF0C
:1001800004680C607047000000230024002500264E
:10019000103A28BF78C1FBD8520728BF30C148BFEA
:1001A0000B607047662908F0BC87642906F0EA8373
:1001B000002070471FB507F00FF804000020002151
:1001C00007F0AAFFE0601FBD10B510BD07F02CF9C5
:1001D0001146FFF7EFFF06F0C7FA07F04AF903B43C
:1001E000FFF7F2FF03BC01F0BBFE000009488047A7
:1001F00009480047FEE7FEE7FEE7FEE7FEE7FEE709
:10020000FEE7FEE7FEE7FEE704480549054A064B20
:10021000704700000B03000831010008680200204D
:100220006808002068040020680400200CB5002045
:10023000019000906C48006840F480306A49086082
:1002400000BF6948006800F4003000900198401C2D
:100250000190009818B90198B0F5A06FF1D16248EB
:10026000006800F4003010B10120009001E000208F
:1002700000900098012843D15C48006840F01000CD
:100280005A4908600846006820F0030008600846E4
:10029000006840F0020008605348406852494860D6
:1002A0000846406848600846406840F480604860FE
:1002B0000846406820F47C1048600846406840F4D6
:1002C000E81048600846006840F08070086000BF91
:1002D0004548006800F000700028F9D042484068A6
:1002E00020F00300404948600846406840F00200A2
:1002F000486000BF3C48406800F00C000828F9D175
:100300000CBD10B5FFF792FF10BD10B53648006860
:1003100040F001003449086008464068344908400C
:100320003149486008460068324908402E49086053
:100330000846006820F4802008600846406820F4E1
:10034000FE0048604FF41F008860FFF7DAFF4FF0AF
:1003500000602949086010BD10B50021002000226E
:10036000214B5B6803F00C0121B1042906D0082958
:1003700028D107E0214B224C236027E01F4B204C63
:10038000236023E0184B5B6803F47010164B5B6826
:1003900003F48032022303EB904022B9194B43430C
:1003A000174C23600DE0104B5B6803F4003323B15E
:1003B000144B4343124C236003E0104B4343104C57
:1003C000236003E00D4B0E4C236000BF00BF064BC3
:1003D0005B68C3F303130C4CE15C094B1B68CB4017
:1003E000074C236010BD00000010024000200240B6
:1003F0000000FFF8FFFFF6FE08ED00E000127A00B3
:100400000000002000093D000400002031490143A4
:10041000314A1160704770B5002100230F22C47863
:1004200004B32D4C246804F4E064C4F5E064210AAC
:10043000C1F10403CA40447804FA03F184781440FB
:1004400021430901254C0678A155047804F01F05C5
:100450000124AC4005786D11AD0005F1E025C5F82B
:10046000004109E0047804F01F050124AC401C4D54
:100470000678761145F8264070BD1A4A0A400243B4
:10048000154B1B1F1A60704739B1134A121D1268B1
:100490000243114B1B1D1A6006E00F4A121D126821
:1004A00082430D4B1B1D1A607047042808D14FF082
:1004B000E021096941F004014FF0E022116107E0F9
:1004C0004FF0E021096921F004014FF0E0221161B1
:1004D000704700000000FA050CED00E000E400E0C9
:1004E00080E100E080FFFF1F10B50446CC48844245
:1004F00008D10121042000F02DFB0021042000F090
:1005000029FB46E0C748844208D10121082000F0B9
:1005100021FB0021082000F01DFB3AE0C248844284
:1005200008D10121102000F015FB0021102000F05F
:1005300011FB2EE0BD48844208D10121202000F0AB
:1005400009FB0021202000F005FB22E0B84884428E
:1005500008D10121402000F0FDFA0021402000F0E8
:10056000F9FA16E0B348844208D10121802000F056
:10057000F1FA0021802000F0EDFA0AE0AE48844252
:1005800007D10121801500F0E5FA0021A01500F047
:10059000E1FA10BD10B50121084600F0DBFA002198
:1005A000012000F0D7FA10BD2DE9F04102460025E8
:1005B0000026002000230024002791F803C00CF03F
:1005C0000F0591F803C00CF0100CBCF1000F03D024
:1005D00091F802C04CEA050591F800C0BCF1000F8B
:1005E00031D0146800202BE04FF0010C0CFA00F31E
:1005F000B1F800C00CEA03069E4220D183004FF000
:100600000F0C0CFA03F7BC4305FA03FC4CEA040494
:1006100091F803C0BCF1280F06D14FF0010C0CFA81
:1006200000FCC2F814C00AE091F803C0BCF1480F06
:1006300005D14FF0010C0CFA00FCC2F810C0401CB0
:100640000828D1D31460B1F800C0BCF1FF0F34DD2D
:10065000546800202EE000F1080C4FF0010808FA61
:100660000CF3B1F800C00CEA03069E4221D18300CE
:100670004FF00F0C0CFA03F7BC4305FA03FC4CEAED
:10068000040491F803C0BCF1280F05D100F1080C57
:1006900008FA0CF8C2F8148091F803C0BCF1480FB6
:1006A00007D100F1080C4FF0010808FA0CF8C2F865
:1006B0001080401C0828CED35460BDE8F0814FF66E
:1006C000FF710180022181700421C17070470246D0
:1006D000002093680B400BB1012000E00020704720
:1006E0000146886880B2704702460020D3680B40FC
:1006F0000BB1012000E0002070470146C86880B2BD
:10070000704701617047416170470AB1016100E0C3
:1007100041617047C16070474FF480320A43826183
:100720008161826182698269704702460020434B81
:1007300018684FF68073184040EA021008433F4B98
:10074000186070473E49C8617047F0B50A460023FB
:1007500000240021002500F00046B6F1004F02D130
:10076000364EF16901E0354E7168C0F3034583B23E
:1007700000F44016B6F5401F08D121F070612F4EED
:10078000766826F070662D4F7E6012E000F48016C9
:10079000B6F5801F06D1032606FA05F4A14341F001
:1007A000706106E0460D360103FA06F6B14341F0EA
:1007B000706122B1460D360103FA06F6314300F0AE
:1007C0000046B6F1004F02D11C4EF16101E01B4E14
:1007D0007160F0BD30B500228B071C0F0F2303FAA8
:1007E00004F2164B08338C1053F824309343134C07
:1007F00008348D1044F8253023468C1053F82430EB
:100800008C07240F00FA04F423430C4C08348D1099
:1008100044F8253030BD0A49DC31086070470000DB
:1008200000080140000C014000100140001401408C
:1008300000180140001C0140002001400000014060
:1008400000002042DF48006840F00100DD490860F8
:1008500008464068DC490840DA49486008460068B4
:10086000DA490840D74908600846006820F480202B
:1008700008600846406820F4FE0048604FF41F00FE
:1008800088607047CF49096821F48031CD4A1160F2
:100890001146096821F480211160B0F5803F03D032
:1008A000B0F5802F0ED106E0C649096841F48031C9
:1008B000C44A116007E0C349096841F4A021C14A54
:1008C000116000E000BF00BF704710B50146002274
:1008D000002300204A11012A02D1BA4C236806E005
:1008E000022A02D1B74C236A01E0B64C636A01F0D8
:1008F0001F02012494401C400CB1012000E00020A4
:1009000010BD38B5002000900024002500BF312024
:10091000FFF7DBFF05460098401C00900098B0F5FB
:10092000A06F01D0002DF2D03120FFF7CEFF08B12B
:10093000012400E00024204638BD01460020A14AE1
:10094000106820F0F80040EAC10010607047A0492C
:1009500008607047024600209A4B586820F47C10CB
:1009600042EA01031843974B58607047984908665C
:10097000704701460020934A506820F00300084366
:10098000506070478F48406800F00C007047014687
:1009900000208C4A506820F0F000084350607047F7
:1009A00001460020874A506820F4E0600843506008
:1009B000704701460020834A506820F4605040EAA6
:1009C000C1005060704729B17E4A527A02437D4B84
:1009D0005A7204E07B4A527A82437A4B5A727047C9
:1009E0007B49D8310860704701460020754A50683D
:1009F00020F440400843506070470021714A203283
:100A00001170704A82F82010012802D004280AD1FF
:100A100004E001216B4A2032117005E00521694A8A
:100A20002032117000E000BF00BF704769490860C4
:100A300070476449096A0143624A11627047654917
:100A400044390860704730B500210022002400239B
:100A50005C4D6D6805F00C0121B1042905D0082911
:100A600023D105E05C4D056022E05B4D05601FE091
:100A7000544D6D6805F47012524D6D6805F4803464
:100A8000022505EB92421CB9544D554305600BE01D
:100A90004C4D6D6805F400351DB1504D5543056052
:100AA00002E04D4D5543056002E04B4D056000BF2F
:100AB00000BF444D6D6805F0F0010909484D6B5CBD
:100AC0000568DD4045603F4D6D6805F4E061090A49
:100AD000434D6B5C4568DD4085603A4D6D6805F4BB
:100AE0006051C90A3E4D6B5C4568DD40C560354DBF
:100AF0006D6805F44041890B3A4D6B5CC568B5FBE8
:100B0000F3F5056130BD29B12E4A526902432D4BE0
:100B10005A6104E02B4A526982432A4B5A6170475A
:100B200029B1284A92690243264B9A6104E0254A7A
:100B300092698243234B9A61704729B1214AD26955
:100B40000243204BDA6104E01E4AD26982431D4B06
:100B5000DA61704729B11B4AD2680243194BDA6047
:100B600004E0184AD2688243164BDA60704729B114
:100B7000144A12690243134B1A6104E0114A1269C4
:100B80008243104B1A617047124940390860704720
:100B90000F49C86470470B49C87170470948406ADB
:100BA00040F0807007494862704701460020054ABE
:100BB00092680A400AB1012000E000207047014914
:100BC00088727047001002400000FFF8FFFFF6FE39
:100BD000000042428004424200127A0000093D00B7
:100BE000140000202400002010B50446FE48844272
:100BF00008D10121C014FFF7ADFF0021E014FFF779
:100C0000A9FFC4E0B4F1804F08D101210846FFF7E5
:100C1000AEFF00210120FFF7AAFFB8E0F3488442AD
:100C200008D101210220FFF7A2FF00210220FFF7D7
:100C30009EFFACE0EE48844208D101210420FFF77A
:100C400096FF00210420FFF792FFA0E0E9488442CC
:100C500008D101210820FFF78AFF00210820FFF7B3
:100C600086FF94E0E448844208D101211020FFF778
:100C70007EFF00211020FFF77AFF88E0DF488442E2
:100C800008D101212020FFF772FF00212020FFF76B
:100C90006EFF7CE0DA48844208D101214014FFF75E
:100CA00059FF00216014FFF755FF70E0D5488442DA
:100CB00009D10121C804FFF74DFF00214FF40020A6
:100CC000FFF748FF63E0D048844209D101210805BD
:100CD000FFF740FF00214FF48010FFF73BFF56E085
:100CE000CA48844209D101214805FFF733FF00219A
:100CF0004FF40010FFF72EFF49E0C548844208D1A9
:100D000001214020FFF733FF00214020FFF72FFF94
:100D10003DE0C048844208D101218020FFF727FF31
:100D200000218020FFF723FF31E0BB48844208D137
:100D300001218015FFF71BFF0021A015FFF717FF0A
:100D400025E0B648844209D101210804FFF702FFDB
:100D500000214FF48030FFF7FDFE18E0B0488442D8
:100D600009D101214804FFF7F5FE00214FF40030BE
:100D7000FFF7F0FE0BE0AB48844208D10121880464
:100D8000FFF7E8FE00214FF48020FFF7E3FE10BDDF
:100D900000220288944B98420ED0994B98420BD077
:100DA000B0F1804F08D0914B984205D0904B9842BB
:100DB00002D0904B984204D14FF68F731A404B8863
:100DC0001A438D4B984207D08C4B984204D04FF673
:100DD000FF431A40CB881A4302808B8883850B8897
:100DE0000385814B98420BD0854B984208D08B4BA2
:100DF000984205D08A4B984202D08A4B984201D142
:100E00000B7A038601238382704770B50024002289
:100E10000023058C4FF6FE7635400584028C8388CE
:100E2000048B4FF68F752C40B51E2C400D882C433B
:100E3000751E2A400D892A434D882A436A4DA842CF
:100E40000BD06F4DA84208D0744DA84205D0744D08
:100E5000A84202D0734DA84213D14FF6F7752A402D
:100E60004D892A434FF6FB752A408D882A434FF659
:100E7000FF652B404FF6FF552B408D892B43CD89C5
:100E80002B4383800483CD888586028470BD70B532
:100E9000002400220023058C4FF6EF7635400584B0
:100EA000028C8388048B48F6FF752C404FF6FF4573
:100EB0002C400D884FF6FF7606EA05252C434FF6A9
:100EC000DF752A400D8906EA05152A434D8806EA92
:100ED00005152A43444DA84202D0494DA8421DD1D0
:100EE0004FF67F752A404D894FF6FF7606EA0515C5
:100EF0002A434FF6BF752A408D8806EA05152A4316
:100F00004FF6FF352B404FF2FF752B408D8906EAD7
:100F100085052B43CD8906EA85052B438380048311
:100F2000CD880587028470BD70B50024002200239F
:100F3000058C4FF6FF6635400584028C8388848BD0
:100F40004FF68F752C404FF6FC752C400D882C43C6
:100F50004FF6FF552A400D894FF6FF7606EA052524
:100F60002A434D8806EA05252A431F4DA84202D090
:100F7000234DA8421DD14FF2FF752A404D894FF6EF
:100F8000FF7606EA05252A434FF6FF352A408D886D
:100F900006EA05252A434EF6FF752B404DF6FF75F0
:100FA0002B408D8906EA05152B43CD8906EA0515E8
:100FB0002B4383808483CD888587028470BD70B580
:100FC000002200230024058C4EF6FF763540058470
:100FD000038C8488828B48F6FF752A404FF6FF45C4
:100FE0002A400D8820E00000002C01400004004051
:100FF00000080040000C00400010004000140040B9
:1010000000340140004C01400050014000540140B8
:1010100000180040001C004000200040004001403B
:1010200000440140004801404FF6FF7606EA0525DE
:101030002A434DF6FF752B400D8906EA05352B43F3
:101040004D8806EA05352B43FA4DA84202D0FA4DE9
:10105000A84208D14BF6FF752C408D894FF6FF76DC
:1010600006EA85152C4384808283CD88A0F8405001
:10107000038470BD828B4FF2FF331A408283828BD0
:101080004FF6FF7303EA01231A4382837047F0B5DA
:101090000C461546002200210026078C4EF6FF7CE8
:1010A00007EA0C070784828B018C4FF6FF7707EA6B
:1010B000043640F6FF473A404FF6FF7707EA052728
:1010C0003A434FF6FF7707EA03373A43D94FB8421E
:1010D0000ED0D94FB8420BD0B0F1804F08D0D74FC7
:1010E000B84205D0D64FB84202D0D64FB84206D14A
:1010F0004DF6FF77394046F48057394305E047F60F
:10110000FF57394044F48057394382830184F0BD4E
:10111000828B4FF6F3731A408283828B0A43828359
:101120007047F0B50C461546002200210026078CBA
:101130004FF6FF6C07EA0C070784828B018C4FF691
:10114000FF7707EA04264FF60C773A404FF6FF7711
:1011500007EA03172F433A43B64FB8420ED0B64FB3
:10116000B8420BD0B0F1804F08D0B44FB84205D090
:10117000B34FB84202D0B34FB84206D14FF6FF5733
:10118000394046F48077394305E04FF2FF57394044
:1011900044F48077394382830184F0BD028B4FF29F
:1011A000FF331A400283028B4FF6FF7303EA0123D9
:1011B0001A4302837047F0B50C4615460022002101
:1011C0000026078C4FF6EF7C07EA0C070784028B9A
:1011D000018C4FF6FF7707EA041640F6FF473A40C6
:1011E0004FF6FF7707EA03373A434FF6FF7707EAF0
:1011F00005273A438F4FB8420ED08F4FB8420BD0DD
:10120000B0F1804F08D08D4FB84205D08C4FB84216
:1012100002D08C4FB84206D14FF6DF77394046F006
:101220001007394305E04FF65F77394044F0100767
:10123000394302830184F0BD028B4FF6F3731A40E9
:101240000283028B0A4302837047F0B50C461546B1
:1012500000220021068C4FF6FE773E400684028B6A
:10126000018C4FF60C7632407E1C06EA03162E43A4
:101270003243704EB0420ED06F4EB0420BD0B0F140
:10128000804F08D06D4EB04205D06D4EB04202D0B6
:101290006C4EB04206D14FF6FD76314044F0010667
:1012A000314305E04FF6F576314044F00106314315
:1012B00002830184F0BD70B505460C465D48854249
:1012C0000ED05D4885420BD0B5F1804F08D05B4809
:1012D000854205D05A48854202D05A48854200D1FD
:1012E00000E000BF208850B92389A2886188284681
:1012F000FFF7ABFFE1882846FFF79EFF25E0208837
:1013000004280AD12389A28861882846FFF753FF61
:10131000E1882846FFF742FF17E0208808280AD115
:101320002389A28861882846FFF7FBFEE1882846CA
:10133000FFF7EEFE09E02389A28861882846FFF7BF
:10134000A6FEE1882846FFF795FE70BD2DE9F04125
:1013500005460C4600260127608808B9022600E0F1
:101360000026A088012801D1022700E0012720885B
:10137000A0B92389A28861882846FFF766FFE18823
:101380002846FFF759FF23893A4631462846FFF79A
:1013900012FFE1882846FFF701FF13E02389A288A6
:1013A00061882846FFF707FFE1882846FFF7F6FE29
:1013B00023893A4631462846FFF747FFE188284609
:1013C000FFF73AFFBDE8F0810A884B881A438B8803
:1013D0001A43CB881A430B891A434B891A438B89CA
:1013E0001A43A0F8442070474FF6FF718180002116
:1013F0000180C180418001727047002101804180DD
:101400008180C180018141818181C181704700213A
:1014100001804180012181800021C18001817047CC
:101420000021018041808180C180018141818181D1
:1014300070470000002C01400034014000040040CF
:1014400000080040000C004021B1028842F0010277
:10145000028004E002884FF6FE731A400280704753
:1014600031B1B0F8442042F40042A0F8442005E035
:10147000B0F84420C2F30E02A0F8442070471AB11D
:1014800083890B43838102E083898B438381704787
:101490008182704741EA0203A0F8483070471AB1D0
:1014A00083890B43838102E083898B438381704767
:1014B00001894FF6F8721140018170470A460021F8
:1014C00001894FF68F73194011430181704730B580
:1014D00004460D4629462046FFF7F0FF208940F0DC
:1014E0000700208130BD2DE9F04104460D46164627
:1014F0001F46602D06D13B46012231462046FFF7AC
:101500005AFE05E03B46012231462046FFF79DFE8C
:1015100029462046FFF7D2FF208940F007002081AE
:10152000BDE8F08130B50C4600210189C9B24FF603
:10153000FF7505EA0325154325432943018130BD85
:101540002DE9F04105460E461746984600244346CD
:101550003A4631462846FFF7E5FF2C894FF6F870EA
:10156000044044F007044FF68F70044044F07004C8
:101570002C81BDE8F081F0B504460D4616461F46A5
:101580003B46324629462046FFF7CCFF208940F4EF
:1015900080402081F0BD0185828270470A4600218B
:1015A00001884FF68F731940114301807047F0B5E1
:1015B0000C4615461E460021002200230189028B9D
:1015C000038C4FF6F877394021434FF6FC473A40F9
:1015D00040F201173A434FF6DD773B404FF6FF7775
:1015E00007EA06172F433B43018102830384F0BDC2
:1015F0000A460021018B4FF68F7319401143018376
:1016000070470A460021018B48F6FF7319404FF6D8
:10161000FF7303EA02231943018370470A4600213E
:10162000818B4FF68F7319401143818370470A46AF
:101630000021818B48F6FF7319404FF6FF7303EAD0
:10164000022319438183704721B1028842F080024E
:10165000028004E002884FF67F731A4002807047D0
:1016600021B1828842F00402828004E082884FF631
:10167000FB731A408280704721B1828842F00802D1
:10168000828004E082884FF6F7731A4082807047A8
:1016900021B1828842F00102828004E082884FF604
:1016A000FE731A40828070470A460021018B4FF674
:1016B000F77319401143018370470A460021018BDB
:1016C0004FF2FF7319404FF6FF7303EA02231943E9
:1016D000018370470A460021818B4FF6F77319404A
:1016E0001143818370470A460021818B4FF2FF73BB
:1016F00019404FF6FF7303EA0223194381837047B1
:101700000A460021018B4FF6FB73194011430183F8
:1017100070470A460021018B4FF6FF3319404FF600
:10172000FF7303EA02231943018370470A4600212D
:10173000818B4FF6FB7319401143818370470A4632
:101740000021818B4FF6FF3319404FF6FF7303EAF8
:1017500002231943818370470A460021018B4FF60B
:101760007F7319401143018370470A460021018BA2
:10177000C1F30E014FF6FF7303EA022319430183FD
:1017800070470A460021818B4FF67F731940114341
:10179000818370470A460021818BC1F30E014FF609
:1017A000FF7303EA02231943818370470A4600212D
:1017B000018C4FF6FD7319401143018470470A46AE
:1017C0000021018C4FF6F7731940114301847047D3
:1017D0000A460021018C4FF6DF7319404FF6FF7364
:1017E00003EA02131943018470470A460021018C61
:1017F0004FF67F7319404FF6FF7303EA0213194344
:10180000018470470A460021018C4FF6FF531940AE
:101810004FF6FF7303EA02231943018470470A4617
:101820000021018C4FF2FF7319404FF6FF7303EA5A
:1018300002231943018470470A460021018C4DF6AA
:10184000FF7319404FF6FF7303EA02331943018413
:10185000704730B5002301248C40A3B2048C9C4314
:101860000484048C02FA01F5ADB22C43048430BD2B
:1018700030B5002304248C40A3B2048C9C43048420
:10188000048C02FA01F5ADB22C43048430BD70B56E
:101890000346002000241846183001258D40ACB2C4
:1018A0001D8CA5431D8409B1082909D100EB6100F5
:1018B000056825F0700505600568154305600EE0B4
:1018C0000D1FC5F34E052844056825F4E045056065
:1018D00005684FF6FF7606EA02263543056070BDBF
:1018E00021B1028842F00202028004E002884FF631
:1018F000FD731A400280704721B1028842F0040251
:10190000028004E002884FF6FB731A4002807047A1
:1019100021B1828842F08002828004E082884FF602
:101920007F731A408280704702884FF6F7731A401F
:10193000028002880A430280704782884FF68F73C4
:101940001A40828082880A438280704702894FF65B
:10195000F8731A40028102890A43028170470289A2
:101960004FF67F731A40028102890A430281704751
:1019700081847047818570478186704701877047F1
:1019800081877047A0F84010704702884FF6FF43E8
:101990001A40028002880A43028070470146888EFE
:1019A00070470146088F70470146888F704701468F
:1019B000B1F8400070470146888C70470146088D99
:1019C000704702460020138A0B400BB1012000E053
:1019D00000207047CA430282704730B5024600209B
:1019E00000230024158A05EA0103958905EA01040C
:1019F00013B10CB1012000E0002030BDCA430282C7
:101A00007047000010B50446FB48844209D101210B
:101A10008803FFF79FF800214FF48040FFF79AF802
:101A200032E0F648844209D101214804FFF79FF8CB
:101A300000214FF40030FFF79AF825E0F048844287
:101A400009D101218804FFF792F800214FF480208A
:101A5000FFF78DF818E0EB48844209D10121C80452
:101A6000FFF785F800214FF40020FFF780F80BE026
:101A7000E548844208D101210805FFF778F80021E4
:101A80004FF48010FFF773F810BD2DE9F04786B0D2
:101A900005460E460024A24600BFA1460027B08995
:101AA00000B100BF2F462C8A4CF6FF700440F0882E
:101AB00004432C82AC894EF6F3100440B08831897F
:101AC0000843718908430443AC81AC8A4FF6FF4058
:101AD0000440B0890443AC8201A8FEF7B4FFC648B5
:101AE000874202D1DDF810A001E0DDF80CA0A88942
:101AF00000F4004040B10AEBCA0000EB0A10316864
:101B00004900B0FBF1F807E00AEBCA0000EB0A104D
:101B100031688900B0FBF1F86420B8FBF0F00401F3
:101B20002009642101FB1089A88900F4004040B11C
:101B3000322000EBC900B0FBF1F000F007000443D5
:101B400008E0322000EB09106421B0FBF1F000F056
:101B50000F0004432C8106B0BDE8F0874FF4165106
:101B6000016000218180C18001810C21418100211F
:101B70008181704710B502460020108A4FF2FF03A2
:101B800018400B884C8823438C882343CC882343FC
:101B90001843108210BD0021018041808180C180E6
:101BA000704721B1828942F40052828104E0828927
:101BB0004DF6FF731A4082817047F0B5034600244A
:101BC00000260025002040F66A17B94200D100BF68
:101BD0001846C1F3421401F01F06012707FA06F563
:101BE000012C01D10C3004E0022C01D1103000E0B6
:101BF00014301AB107682F43076002E00768AF434B
:101C00000760F0BD1AB1838A0B43838202E0838AA6
:101C10008B4383827047028A4FF6F0731A40028228
:101C2000028A0A430282704782894FF2FF731A4088
:101C3000828182890A438281704721B1828942F080
:101C40000202828104E082894FF6FD731A4082818C
:101C50007047028A4FF6DF731A400282028A0A43F3
:101C60000282704721B1028A42F48042028204E07B
:101C7000028A4BF6FF731A4002827047C1F30802D2
:101C80008280704701468888C0F3080070478189C8
:101C900041F0010181817047028BD2B20283028B35
:101CA00042EA012202837047028B02F47F420283E0
:101CB000028B0A430283704721B1828A42F02002DC
:101CC000828204E0828A4FF6DF731A408282704774
:101CD00021B1828A42F01002828204E0828A4FF6A9
:101CE000EF731A408282704721B1828A42F0080263
:101CF000828204E0828A4FF6F7731A40828270472C
:101D000021B1828942F40042828103E08289C2F3D8
:101D10000E028281704721B1828A42F4006282827F
:101D200004E0828A4FF2FF731A4082827047828AEF
:101D30004FF6FB731A408282828A0A43828270477E
:101D400021B1828A42F00202828204E0828A4FF646
:101D5000FD731A408282704702460020B1F5007F71
:101D600000D100BF13880B400BB1012000E0002020
:101D7000704701F40072B2F5007F00D100BFCA4382
:101D80000280704770B50246002400230025002021
:101D900040F66A16B14200D100BFC1F3421501F00E
:101DA0001F03012606FA03F3012D02D19689334061
:101DB00006E0022D02D1168A334001E0968A3340B4
:101DC0000C12012606FA04F41688344013B10CB143
:101DD000012000E0002070BD10B50022002340F675
:101DE0006A14A14200D100BF0A1201249440A3B298
:101DF000DC43048010BD0000003801400044004076
:101E000000480040004C00400050004070B54820A1
:101E100000F01CF900F064F800F02EF84FF4E13007
:101E200000F060F800F03AFF002140F60F6000F08B
:101E30007DFA00F038FB47F230504FF08041888443
:101E400000F07EFB47F230500949088064210846C3
:101E500000F0CEFA00F0EEFA642000F011F94FF431
:101E6000FA752C4603480580001D048070BD0000F3
:101E7000240800403C04004008B501211020FEF772
:101E80004FFE4FF40050ADF8000010208DF8030015
:101E900003208DF8020069460F48FEF785FB08BD58
:101EA00070B504460D480068401C0C490860A0420B
:101EB00010D14FF400510848FEF709FCC0F10100B1
:101EC000C5B22A464FF400510348FEF71EFC00201D
:101ED0000249086070BD0000001001402800002089
:101EE0007047000010B586B00446012144F204009A
:101EF000FEF716FE4FF40070ADF8140018208DF8B0
:101F0000170003208DF8160005A94B48FEF74CFB7F
:101F10004FF48060ADF8140004208DF8170005A977
:101F20004548FEF741FB01940020ADF80800ADF8EC
:101F30000A00ADF80C00ADF810000C20ADF80E0052
:101F400001A93E48FFF7A1FD012240F225513B487F
:101F5000FFF733FE01213948FFF723FE06B010BD1D
:101F600000BF704700BF354A128802F04002002AC5
:101F7000F9D0C2B2314B1B1D1A80704710B5044610
:101F800000BF20212D48FFF7E7FE0028F9D02B489D
:101F9000FFF778FE10BD70B504460D464021274876
:101FA000FFF7E7FE80212548FFF716FF13E02178B1
:101FB0002248FFF763FE00BF40212048FFF7CCFE18
:101FC0000128F9D140211D48FFF7D3FE80211B488D
:101FD000FFF702FF641C281EA5F10105E7D170BDC3
:101FE0000022174B1A60174A1160174A1060704799
:101FF00010B540F225511148FFF7C4FED8B10F4883
:10200000FFF740FEC4B20F4800680D4909688842D6
:102010000CD90D48006804700B480068401C0A4940
:10202000086007480068401C0549086040F22551D7
:102030000248FFF7D1FE10BD000801400038014002
:1020400030000020340000202C00002010B5044691
:102050006FF00400FEF729FAE11704EB5171C1F3A8
:10206000C701234A11701046007800EB4001C1EB14
:10207000C0104FF6FF7101EAC0001E49088010BD74
:1020800001461C4A12884A434FF0E0235A6100225D
:102090009A6101221A6100BF4FF0E022106900F03E
:1020A00001021AB100F48032002AF5D000224FF06C
:1020B000E0231A619A61704701460D4A12784A433B
:1020C0004FF0E0235A6100229A6101221A6100BF99
:1020D0004FF0E022106900F001021AB100F48032E2
:1020E000002AF5D000224FF0E0231A619A61704770
:1020F0003C0000203E000020002001E0411CC8B24E
:102100000A28FBDB704710B54FF400618148FEF7E9
:10211000F8FA4FF480617F48FEF7F3FAFFF7ECFF1F
:102120004FF400617B48FEF7EEFAFFF7E5FF4FF44E
:1021300080617848FEF7E7FAFFF7DEFF10BD10B5C3
:102140004FF400617348FEF7DEFA4FF48061714886
:10215000FEF7D7FAFFF7D0FF4FF400616D48FEF7A6
:10216000D0FA10BD70B50446002528E004F08000C8
:1021700028B14FF400616748FEF7C3FA04E04FF45A
:1021800000616448FEF7BFFAFFF7B6FF4FF48061C5
:102190006048FEF7B6FAFFF7AFFF4FF480615D4885
:1021A000FEF7B1FA072D04D14FF400615948FEF74C
:1021B000A8FA6006040EFFF79FFF681CC5B2082D41
:1021C000D4DB70BD10B54FF400615248FEF79BFAA6
:1021D000FFF792FF4FF480614E48FEF792FAFFF747
:1021E0008BFF4FF480614B48FEF78DFAFFF784FFB9
:1021F0004FF400614748FEF784FA10BD10B54FF464
:1022000000614448FEF77DFAFFF776FF4FF48061E6
:102210004048FEF776FAFFF76FFF4FF480613D48C4
:10222000FEF771FAFFF768FF10BD70B50546002490
:10223000002619E06006040E4FF480613548FEF771
:1022400060FAFFF759FF4FF400613248FEF73FFA9A
:1022500008B1601CC4B24FF480612E48FEF753FAF7
:10226000FFF74AFF701CC6B2082EE3DB15B9FFF773
:10227000C5FF01E0FFF7A6FF204670BD10B54FF483
:1022800000612448FEF73DFAFFF736FF4FF4806106
:102290002048FEF736FAFFF72FFF4FF400611D4884
:1022A000FEF715FA08B1012400E000244FF4806124
:1022B0001848FEF728FAFFF71FFF204610BD08B5A3
:1022C00015A1194800F020FC01210820FEF728FC88
:1022D0004FF44060ADF8000003208DF80200142098
:1022E0008DF8030069460B48FEF75EF9FFF727FFFC
:1022F00008BD70B50446FFF7E2FFFFF704FF204674
:10230000FFF730FFFFF7BAFF0546FFF718FF284633
:1023100070BD0000000C014049494320496E6974BA
:102320002E2E0D0A000000000044004030B589B098
:1023300005460C4601210220FEF7FFFB681E80B215
:10234000ADF80800A0B2ADF804000020ADF80A0016
:10235000ADF8060001A9C048FEF71AFD0121BE48EC
:10236000FFF738FB01221146BB48FFF788F801212F
:102370000820FEF7D5FB0320ADF8100018208DF8DB
:10238000130003208DF8120004A9B448FEF70CF9DD
:102390006020ADF814000120ADF816000020ADF863
:1023A0001A00ADF81C0005A9AB48FEF7BDFD0821D9
:1023B000A948FFF727FA6020ADF814000120ADF816
:1023C00016000020ADF81A00ADF81C0005A9A248BF
:1023D000FEF7F5FD0821A048FFF72EFA01219E48DF
:1023E000FFF732F901219C48FFF72EF809B030BD04
:1023F0007FB505460C466020ADF800000120ADF821
:102400000200ADF8065069469348FEF78DFD08219D
:102410009148FFF7F7F9ADF8064069468E48FEF798
:10242000CEFD08218C48FFF707FA01218A48FFF703
:102430000BF97FBD1FB501211020FEF77EFB42F294
:102440000F70ADF8080040F2CF20ADF80400002076
:10245000ADF80A00ADF806008DF80C0001A980481F
:10246000FEF796FC01217E48FFF7B4FA01221146DF
:102470007B48FFF704F84FF44070FDF7C7FF3620A4
:102480008DF8000005208DF8010000208DF8020075
:1024900001208DF803006846FDF7BDFF012170485B
:1024A000FEF7D2FF1FBD00B587B001210846FEF739
:1024B00044FB01210420FEF733FB0320ADF80000AC
:1024C00004208DF8030069466648FEF76DF804A8FD
:1024D000FEF78AFF0020ADF810004EF66020ADF840
:1024E00014000020ADF81600ADF8120004A94FF05A
:1024F0008040FEF74DFC00231A4603214FF0804038
:10250000FFF755F801A8FEF782FF0A20ADF80C008E
:1025100001A94007FEF7CFFE01218807FFF75AFA0D
:10252000012211469007FEF7AAFF00214FF08040DC
:10253000FFF71EFA01218807FEF786FF07B000BDEE
:1025400000B587B001210420FEF7F7FA0121082029
:10255000FEF7E6FAC020ADF8000004208DF8030075
:1025600069463E48FEF720F804A8FEF73DFF00202C
:10257000ADF810004EF66020ADF814000020ADF864
:102580001600ADF8120004A93748FEF701FC00233D
:102590001A4603213448FFF70AF801A8FEF737FF6F
:1025A0000A20ADF80C0001A92F48FEF784FE012196
:1025B0002D48FFF70FFA012211462B48FEF75FFF67
:1025C00000212948FFF7D4F901212748FEF73CFFF5
:1025D00007B000BD0146022904D003290CD004290C
:1025E0001ED113E04FF08042928C10B247F230526D
:1025F0004FF080439A8415E0174A2432128810B2B3
:1026000047F23052144B24331A800BE0164A24321E
:10261000128810B247F23052134B24331A8001E073
:10262000002000BF00BF70470F48103000880E48E0
:102630001030008820F001000B49103108807047ED
:102640004FF08040008A4FF08040008A20F0010067
:102650004FF080410882704700040040000C0140A8
:1026600000100040000801400008004070472DE9BC
:10267000FC5F04460D462E1B3648006806F074FBCE
:10268000834635480168584606F0CEFB81463348FC
:10269000006806F069FB009031480168009806F078
:1026A000C3FB8346304606F05FFB00902D4801686F
:1026B000009806F0B9FB5946019006F0BDFC824631
:1026C000494606F0B1F9804606F012FB074623485A
:1026D000006820490860214806603846BDE8FC9F34
:1026E0002DE9FC5F04460D462E1B1F48006806F0CE
:1026F0003BFB834618480168584606F095FB814627
:102700001A48006806F030FB0090154801680098F0
:1027100006F08AFB8346304606F026FB00901148FF
:102720000168009806F080FB5946019006F084FC91
:102730008246494606F078F9804606F0D9FA0746FF
:102740000A48006808490860084806603846BDE83D
:10275000FC9F000050000020480000204C0000209A
:1027600044000020400000205800002054000020B9
:102770002DE9F05F01216C48FFF723F900287DD097
:1027800001216948FFF73AF90520FFF789FB02208C
:10279000FFF720FFA0F5EA403038644908600420C4
:1027A000FFF718FFA0F5EA40303861490860084695
:1027B00000685E49096800EB010A0AEBDA70401014
:1027C0004FF4167148434FF41C6190FBF1FB5846DF
:1027D00005F0F2FE8046574A574B05F005FF0646C6
:1027E000564A574B05F000FF044605F0ABFC55492F
:1027F00008600846006806F0EBF8044622460B46DF
:1028000051A1534804F082F848480068002804DACF
:10281000464800684042454908604548006800282D
:1028200004DA43480068404241490860494800686A
:102830004FF41C6148434FF4167190FBF1F42146AC
:102840003A480068FFF713FF4349086041480068B1
:102850004FF41C6148434FF4167190FBF1F421468C
:1028600033480068FFF73CFF3C4908603A4800687D
:1028700010F1030F05DB3848006800E052E0032840
:1028800006DD37480068344909680844344908605F
:102890003248006810F1030F03DB3048006803285A
:1028A00006DD304800682D49096808442D49086054
:1028B0002B48006840F6AC51884203DD40F6B83042
:1028C000274908602748006840F6AC51884203DD7C
:1028D00040F6B8302349086040F2DC5020490860D7
:1028E000204908601E4800881F4908801D4800884C
:1028F000091D0880FFF7BAFE0C4800684FF41671F6
:1029000048434FF41C6190FBF1F0184908600848F7
:1029100000684FF4167148434FF41C6190FBF1F0CE
:1029200013490860BDE8F09F001000405C000020E3
:1029300060000020A4703D0AD7A3B03F6F1283C08F
:10294000CA2109408000002025322E326600000096
:102950008D000020740000206C000020700000201A
:1029600064000020680000203C0400407800002043
:102970007C00002010B586B0044601210420FEF73B
:10298000CFF801214804FEF7D8F80420ADF8140070
:1029900018208DF8170003208DF8160005A9BA48F5
:1029A000FDF702FE0820ADF8140004208DF8170092
:1029B00005A9B548FDF7F8FD01940020ADF8080021
:1029C000ADF80A00ADF80C00ADF810000C20ADF821
:1029D0000E0001A9AD48FFF758F84FF4E060FDF78D
:1029E00015FD26208DF8000000208DF801008DF8DF
:1029F000020001208DF803006846FDF70CFD01225E
:102A000040F22551A148FFF7D8F801219F48FFF770
:102A1000C8F806B010BD70B504460D4640219B486D
:102A2000FFF7A7F980219948FFF7D6F913E021783D
:102A30009648FFF723F900BF40219448FFF78CF92F
:102A40000128F9D140219148FFF793F980218F485F
:102A5000FFF7C2F9641C281EA5F10105E7D170BD7E
:102A600010B5044640218948FFF783F98021874843
:102A7000FFF7B2F913E014F8011B8448FFF7FEF8E2
:102A800000BF40218148FFF767F90128F9D14021B3
:102A90007E48FFF76EF980217C48FFF79DF920788A
:102AA0000028E8D110BDF0B503460D4616460027B4
:102AB00029460A2E03D0002008702846F0BD33B9FD
:102AC000302001F8010B002008702846F6E7002BA3
:102AD00003DA2D2001F8010B5B4242F210720DE087
:102AE00093FBF2F404B937B104F1300001F8010BA3
:102AF00004FB123301270A2092FBF0F2002AEFDCDC
:102B0000002008702846D9E70FB470B586B0064695
:102B10000CA8009040215D48FFF72BF980215B480D
:102B2000FFF75AF97BE00B9800785C281CD10B98D2
:102B3000401C0B9000786E2809D072280FD10D210F
:102B40003046FFF79BF80B98401C0B900BE00A21D6
:102B50003046FFF793F80B98401C0B9003E00B985E
:102B6000401C0B9000BF4BE00B980078252840D10B
:102B70000B98401C0B900078642818D0732833D130
:102B8000009810C800900BE021783046FFF776F8E7
:102B900000BF40213046FFF7DFF80028F9D0641C61
:102BA00020780028F0D10B98401C0B9020E0009872
:102BB00020C800900A2201A92846FFF774FF01AC43
:102BC0000BE021783046FFF759F800BF402130462E
:102BD000FFF7C2F80028F9D0641C20780028F0D153
:102BE0000B98401C0B9003E00B98401C0B9000BF0F
:102BF00006E00B9810F8011B0B903046FFF73EF8EB
:102C000000BF40213046FFF7A7F80028F9D0402147
:102C10001E48FFF7AEF880211C48FFF7DDF80B983F
:102C2000007800287FF47FAF06B070BC5DF814FB1D
:102C30000022174B1A60174A1160174A106070473C
:102C400010B540F225511148FFF79CF8D8B10F4854
:102C5000FFF718F8C4B20F4800680D4909688842A8
:102C60000CD90D48006804700B480068401C0A49E4
:102C7000086007480068401C0549086040F225517B
:102C80000248FFF7A9F810BD0008014000440040C9
:102C9000980000209C0000209400002008B501212D
:102CA0000820FDF73DFF4FF47C40ADF800001020F8
:102CB0008DF8030003208DF8020069463748FDF7C0
:102CC00073FC08BD10B504464CB94FF4805133482D
:102CD000FDF717FD4FF400513048FDF714FD012CAE
:102CE00007D161032D48FDF70CFD21032B48FDF7AB
:102CF0000AFD022C07D1E1022848FDF704FD21035B
:102D00002648FDF700FD10BD10B504464CB94FF440
:102D100000412248FDF7F5FC4FF480411F48FDF7C4
:102D2000F2FC012C07D1A1031C48FDF7EAFCE103EA
:102D30001A48FDF7E8FC022C07D161031748FDF79C
:102D4000E2FCA1031548FDF7DEFC10BD10B5002024
:102D5000FFF7B8FF0020FFF7D7FF10BD10B5012027
:102D6000FFF7B0FF0120FFF7CFFF10BD10B5012026
:102D7000FFF7A8FF0020FFF7C7FF10BD10B5002028
:102D8000FFF7A0FF0120FFF7BFFF10BD10B5022025
:102D9000FFF798FF0220FFF7B7FF10BD000C0140BE
:102DA00008B501210820FDF7BBFE4FF44070ADF8D7
:102DB000000010208DF8030003208DF80200694602
:102DC000F748FDF7F1FB08BD10B5F548001D006898
:102DD00020F47040F249091D08600846006840F080
:102DE000300008600120EF490860EF48D0F82C015E
:102DF00008B9002010BD0120EA49091F0860FFF74B
:102E00005BF90020E849C1F8AC01E6488038006869
:102E100008B10020EEE70120FFF74EF90020E1495C
:102E2000091F08600120E5E710B5DD48001D0068B6
:102E300020F47040DA49091D08600846006840F037
:102E4000300008600020D749091F0860D649C1F842
:102E5000AC010120FFF730F90120D249091F0860B9
:102E6000D149C1F8AC01FFF727F910BD10B5002416
:102E7000CB48001D006820F47040C949091D086056
:102E80000846006840F0800008600120C5490860DD
:102E9000FFF712F90120C449C1F8A801FFF70CF9A6
:102EA0000AE0601CC4B2322C03DDFFF7BDFF002036
:102EB00010BD0120FFF700F9BA48803800680028EB
:102EC000EFD1B849091F08600120F1E710B50020D3
:102ED000B449091F0860B248001D006820F4704022
:102EE000AF49091D08600846006840F030000860DE
:102EF0000020AD49C1F8AC010120FFF7DDF8012049
:102F0000A849091F0860FFF7D7F80020A649C1F8B3
:102F1000A80110BD10B50020A249091F0860A048F3
:102F2000001D006820F470409D49091D0860084696
:102F3000006840F03000086001209B49C1F8AC01F6
:102F4000FFF7BAF801209749091F0860FFF7B4F8A6
:102F500000209549C1F8A80110BD70B504469048FD
:102F6000001D006820F470408D49091D0860084666
:102F7000006840F03000086000208A49091F08609E
:102F8000002516E0E009874908606006040E01206C
:102F9000FFF792F801208449C1F8A801FFF78CF8E7
:102FA00000208049091F08600120FFF785F8681C90
:102FB000C5B2082DE6DB70BD2DE9F04105460E4691
:102FC00017469846FFF700FF10B90120BDE8F081D1
:102FD0006906080EFFF7C1FFFFF748FF18B9FFF7B2
:102FE00023FF0120F2E73046FFF7B7FFFFF73EFF70
:102FF00000240BE018F80400FFF7AFFFFFF736FFDF
:1030000018B9FFF711FF0020E0E7641CBC42F1DBB8
:10301000FFF70AFF0020D9E770B505460024604895
:10302000001D006820F470405D49091D08600846D5
:10303000006840F080000860002617E00020594931
:10304000091F08600220FFF737F801205649C1F830
:10305000A8016006040E53488038006808B1601C5F
:10306000C4B20220FFF728F8701CC6B2082EE5DBB8
:1030700015B1FFF72BFF01E0FFF74CFF204670BDB5
:103080002DE9F04106460F4614461D46FFF79CFE0B
:1030900010B90120BDE8F0817106080EFFF75DFF51
:1030A000FFF7E4FE18B9FFF7BFFE0120F2E738464C
:1030B000FFF753FFFFF7DAFEFFF786FE012101EB72
:1030C0004601C8B2FFF749FFFFF7D0FE0DE0012C23
:1030D00004D10020FFF7A0FF287003E00120FFF7D4
:1030E0009BFF28706D1C601EC4B2002CEFD1FFF74F
:1030F0009BFE0020CEE770B505460E460024FFF784
:1031000063FE2846FFF729FF641CFFF7AFFE304639
:10311000FFF723FF641CFFF7A9FEFFF755FE691CAC
:10312000C8B2FFF71AFF641CFFF7A0FE0020FFF7EC
:1031300073FF0446FFF778FE204670BD2DE9F0418D
:103140000746884615461E460024FFF73DFE3846D2
:10315000FFF703FFFFF78AFE4046FFF7FEFEFFF78B
:1031600085FEFFF731FE791CC8B2FFF7F6FEFFF7C8
:103170007DFE00BF0DE0681EA04204D00120FFF7D5
:103180004BFF305503E00020FFF746FF3055601C31
:10319000C4B2AC42EFDBFFF747FE2046BDE8F0814A
:1031A000000C0140AC812142008021422DE9F04118
:1031B00080460D4616461F460024FFF705FE404692
:1031C000FFF7CBFEFFF752FE2846FFF7C6FEFFF7DC
:1031D0004DFE00BF06E0385DFFF7BFFEFFF746FE7D
:1031E000601CC4B2B442F6DBFFF71EFE0120BDE84E
:1031F000F08170B505460E46144631462846FFF765
:103200007AFF2070012070BD37B504460D4602AB31
:10321000012229462046FFF7C9FF3EBD2DE9F843AC
:103220000746884614461D46089E6A46414638466B
:10323000FFF7DFFF28B3601CFF2101FA00F0C4F1A3
:1032400008012944491EFF220A41104300F0FF09EA
:10325000C5F1080006FA00F0C6B2C4F10700064145
:103260009DF8000000EA090000909DF8000030433E
:1032700000909DF8002041463846FFF7C5FFBDE8A5
:10328000F8830020FBE7F8B506460F4614461D46B6
:103290006A4639463046FFF7ACFF2DB10120A04009
:1032A0009DF80010084305E00120A0409DF80010A3
:1032B00021EA0000C0B200909DF800203946304657
:1032C000FFF7A2FFF8BD0000014691F90020002A97
:1032D00001DD00201EE091F90020002A01DA04201F
:1032E00018E091F90120002A01DD012012E091F996
:1032F0000120002A01DA05200CE091F90220002AC1
:1033000001DD022006E091F90220002A01DA062000
:1033100000E00720704770B505462846FFF7D4FF48
:103320000446E81CFFF7D0FF44EAC00084B2A81DA1
:10333000FFF7CAFF44EA801084B2204670BD70B522
:1033400088B002A905A801F092FF0446072C40D1DD
:1033500001A801F001FA059805F006FD064601995D
:1033600005F062FD054605F0C3FC0590069805F0E2
:10337000FBFC0646019905F057FD054605F0B8FC33
:103380000690079805F0F0FC0646019905F04CFD03
:10339000054605F0ADFC079005A802F078FA6846EE
:1033A00001F0F7F9BDF80010029848430290BDF80B
:1033B0000010039848430390BDF800100498484358
:1033C000049002A802F0F6FAF5A1FE48FFF79CFB74
:1033D00003E0FDA1FB48FFF797FB08B070BD2DE9A6
:1033E000F04304460D46DDE907670021012041E076
:1033F000DFF8E0C33CF81080A0F1010CDFF8D493B3
:1034000029F81C8009F1160C3CF81090A0F1010C71
:10341000DFF8C08308F1160828F81C9008F1160C94
:103420003CF81090A0F1010C08F1160828F81C9047
:1034300008F1160C3CF81090A0F1010C08F11608E8
:1034400028F81C9008F1160C3CF81090A0F1010C23
:1034500008F1160828F81C9008F1160C3CF810909A
:10346000A0F1010C08F1160828F81C9000F1010CDD
:103470000CF0FF000A28BBDBDFF858C3ACF81240A1
:10348000ACF82850ACF83E20ACF85430ACF86A6088
:10349000ACF880700021002008E0DFF838C33CF968
:1034A00010C0614400F1010C0CF0FF000A28F4DBAD
:1034B0004FF00A0C91FBFCFC0FFA8CFCDFF8148334
:1034C000A8F814C0002100200AE0DFF808C30CF1BE
:1034D000160C3CF910C0614400F1010C0CF0FF0027
:1034E0000A28F2DB4FF00A0C91FBFCFC0FFA8CF877
:1034F000DFF8E0C2ACF82A80002100200AE0DFF803
:10350000D4C20CF12C0C3CF910C0614400F1010C48
:103510000CF0FF000A28F2DB4FF00A0C91FBFCFCD8
:103520000FFA8CF8DFF8ACC2ACF840800021002024
:103530000AE0DFF8A0C20CF1420C3CF910C0614473
:1035400000F1010C0CF0FF000A28F2DB4FF00A0C2E
:1035500091FBFCFC0FFA8CF8DFF878C2ACF85680CF
:10356000002100200AE0DFF86CC20CF1580C3CF995
:1035700010C0614400F1010C0CF0FF000A28F2DBDE
:103580004FF00A0C91FBFCFC0FFA8CF8DFF844C2F8
:10359000ACF86C80002100200AE0DFF838C20CF1A2
:1035A0006E0C3CF910C0614400F1010C0CF0FF00FE
:1035B0000A28F2DB4FF00A0C91FBFCFC0FFA8CF8A6
:1035C000DFF810C2ACF88280BDE8F08338B504465D
:1035D000032302226B21D0200094FFF71FFE38BD89
:1035E00038B50446022304221B21D0200094FFF7A3
:1035F00015FE38BD38B50446022304221C21D02014
:103600000094FFF70BFE38BD10B504462346062292
:103610006B21D020FFF737FE10BD10B56E4B012295
:103620007521D020FFF78AFD6B48007810BD10B5DA
:10363000FFF7F3FF682801D1012010BD0020FCE74F
:1036400010B50446234605226A21D020FFF71BFE51
:1036500010BD10B50446234601223721D020FFF7C4
:1036600012FE10BD10B55DA15648FFF74DFAFFF7E9
:1036700066FE0220FFF7AAFF0320FFF7B1FF00203C
:10368000FFF7B8FF0020FFF7BFFF0020FFF7D8FFCC
:103690000020FFF7DEFF10BD38B5002000906B461C
:1036A000012275216820FFF7EBFC9DF800006828D7
:1036B00005D09DF800204EA14248FFF725FA00F002
:1036C00058FDE0B9782000F0BCF9782000F0A0FBAC
:1036D000C82000F07EFC02F03FF84948FFF71BFECF
:1036E000044602F043F840F2731002F080FCC82058
:1036F00002F0F6F9FFF723FE012001F073FD38BD5B
:103700002DE9F04F8DB00AA83E490BAB06AACDE9D2
:1037100000103D493D4802F0C9FD3A48008800F4D8
:10372000807000287CD0069805F01EFB04464FF000
:103730009D4105F0E7F936490860079805F014FB4C
:1037400004464FF09D4105F0DDF9324908600898C4
:1037500005F00AFB04464FF09D4105F0D3F92E49D0
:103760000860099805F000FB04464FF09D4105F004
:10377000C9F92A490860284801684FF0804005F0DF
:1037800053FB019024480168019805F04DFB8246E7
:10379000204801684FF0404005F046FB019040E0B2
:1037A00073657474696E67206269617320737563F1
:1037B00063657366756C6C79202E2E2E2E2E2E0D61
:1037C0000A000000004400404661696C2E2E0D0A7C
:1037D000000000002E0100202001002072756E5FA5
:1037E00073656C665F746573742E2E0D0A0000009D
:1037F00077686F20616D20692025640D0A00000044
:10380000C8000020AC000020A6000020A00000207E
:10381000B8000020BC000020C0000020C400002030
:1038200043E023480168019805F0FEFA83465146BB
:1038300005F002FC81464FF07E5105F0F5F8044694
:1038400005F0C6F8CDE902011A4801684FF0804042
:1038500005F0EAFA834616480168584605F0E4FA8E
:103860008146154801684FF0804005F0DDFA834637
:1038700012480168584605F0D7FA8246494605F0D5
:10388000D3F8044605F0A4F80746DDE9022304F066
:1038900083FB4FF066320A4BCDE9040104F0A4FE2D
:1038A000054604F04FFC074908600DB0BDE8F08FF5
:1038B000BC000020B8000020C0000020C400002090
:1038C00066A64C40B400002038B50446FB4890F88A
:1038D0002400C0B114B10220009001E0002000904B
:1038E000F64A1268D17BF54A526810786B4601227D
:1038F000FFF762FB10B14FF0FF3038BD9DF80010AC
:10390000EE48417423E0ED48807A10B94FF0FF3063
:10391000F3E724B1E948407C08B10020EDE714B199
:103920000120009001E000200090E44A1268D17B61
:10393000E24A526810786B460122FFF73DFB10B156
:103940004FF0FF30D9E79DF80010DC4841740020AB
:10395000D3E738B5002419E0D8480068C07AA042FF
:1039600004D0D6480068407DA04200D10CE0D34985
:10397000496808786B4601222146FFF781FB10B1A8
:103980004FF0FF3038BD00BF601CC4B2CB48406868
:103990000079A042E0DC0020F4E770B504460D4653
:1039A000C6480068C07AA04204D0C4480068407D80
:1039B000A04202D14FF0FF3070BDC048406800798E
:1039C000A04202DC4FF0FF30F6E7BC4949680878B6
:1039D0002B4601222146FFF753FBEDE738B504469D
:1039E000B64890F82300A04201D1002038BD14B1A0
:1039F0003020009001E000200090B048807C20B191
:103A00009DF8000040F002000090AC4890F82200C1
:103A100020B19DF8000040F080000090A74A126895
:103A2000117DA64A526810786B460122FFF7C4FA4E
:103A300010B14FF0FF30D9E7A04880F823400020B4
:103A4000D4E738B5044604F0700010B101200090AE
:103A500005E014B10020009001E040200090974A5A
:103A60001268917C954A526810786B460122FFF7E4
:103A7000A3FA20B1002191488172481E38BD9DF8FB
:103A8000000020F040018D4801730020009004F0F8
:103A9000400020B99DF8000040F00400009004F0C0
:103AA000200020B99DF8000040F00200009004F0D2
:103AB000100020B99DF8000040F00100009004F0D3
:103AC000080020B99DF8000040F0380000907B4AC3
:103AD0001268D17C794A526810786B460122FFF750
:103AE0006BFA20B1002175488172481EC6E724B1E7
:103AF000082C02D00020FFF771FF7048847200216B
:103B000001753220FEF7BCFA0020B7E738B504464D
:103B10006A48807CA04201D1002038BD002C46D0EC
:103B2000664A12681179654A526810786B4601221C
:103B3000FFF7A6FA10B14FF0FF30EEE79DF8000056
:103B400020F0200000905D4A126811795B4A5268AB
:103B500010786B460122FFF72FFA10B14FF0FF30BB
:103B6000DBE70320FEF78CFA02200090534890F820
:103B7000220020B19DF8000040F0800000904F48E6
:103B800090F8230020B19DF8000040F03000009034
:103B90004A4A1268117D494A526810786B460122E0
:103BA000FFF70AFA002851D04FF0FF30B5E7434A3B
:103BB00012681179414A526810786B460122FFF76A
:103BC0005FFA10B14FF0FF30A7E73C48807A00F071
:103BD000010028B19DF8000040F02000009004E0B2
:103BE0009DF8000020F020000090344A12681179FE
:103BF000324A526810786B460122FFF7DDF910B1A6
:103C00004FF0FF3089E70320FEF73AFA2B4890F88F
:103C1000220010B18020009001E000200090274891
:103C200090F8230020B19DF8000040F03000009093
:103C3000224A1268117D214A526810786B4601228F
:103C4000FFF7BAF910B14FF0FF3066E71B488474F4
:103C5000002062E708B51948807A10B94FF0FF30AC
:103C600008BD00200090154A1268D17B134A5268A3
:103C700010786B460122FFF79FF910B14FF0FF302B
:103C8000EEE70E4A126851790C4A526810786B467A
:103C90000122FFF791F910B14FF0FF30E0E7074A3A
:103CA00012681179054A526810786B460122FFF7B5
:103CB00083F928B14FF0FF30D2E70000D800002090
:103CC000F74890F82400002850D00C200090F44AC7
:103CD00012681179F24A526810786B460122FFF798
:103CE0006BF910B14FF0FF30BAE7C0200090EC48FC
:103CF000807A00F0010020B19DF8000040F0200023
:103D00000090E74A12681179E54A526810786B46CC
:103D10000122FFF751F910B14FF0FF30A0E7E04862
:103D2000407C10B10220009001E000200090DC4AAD
:103D30001268D17BDA4A526810786B460122FFF78D
:103D40003BF910B14FF0FF308AE700200090D44AD1
:103D500012685179D24A526810786B460122FFF7F7
:103D60002BF9002852D04FF0FF3079E70420009063
:103D7000CB4A12681179CA4A526810786B46012200
:103D8000FFF71AF910B14FF0FF3069E7C448807CA3
:103D900020B9C348807A00F0010010B9402000909B
:103DA00001E060200090BE4A12681179BC4A526856
:103DB00010786B460122FFF7FFF810B14FF0FF308B
:103DC0004EE7B748407C10B10120009001E0002090
:103DD0000090B34A1268D17BB14A526810786B46A2
:103DE0000122FFF7E9F810B14FF0FF3038E7AC4A95
:103DF00012685179AA4A52681078A94B10330122EF
:103E0000FFF7DAF810B14FF0FF3029E7002027E77D
:103E100070B50446002624F00104A14890F824005F
:103E200008B1002070BD9E48807A10B94FF0FF3075
:103E3000F8E79B48057C807A204099490874084639
:103E4000007CA04202D04FF0FF3600E0002614B9FB
:103E50009348007D18B10120FFF736FD02E00020F5
:103E6000FFF732FD3CB1FFF7F5FE20B18C48057439
:103E70004FF0FF30D6E73046D4E738B504468848DF
:103E8000807A10B94FF0FF3038BDBC2C02DB012026
:103E9000009015E0622C02DB0220009010E02A2C3A
:103EA00002DB032000900BE0142C02DB04200090C6
:103EB00006E00A2C02DB0520009001E006200090BD
:103EC0007748C07A9DF80010884201D10020DBE7D6
:103ED000734A12689178724A526810786B460122D0
:103EE000FFF76AF810B14FF0FF30CDE79DF80010F2
:103EF0006B48C1720020C7E738B50446282C02DDA4
:103F00004FF0FF3038BDDCB90020FFF767FD00201F
:103F10008DF8000007208DF80100614A1268917C3D
:103F20005F4A526810786B460222FFF745F810B1DD
:103F30004FF0FF30E6E70021594801750020E1E726
:103F40000120FFF74BFD20208DF80000012C06D149
:103F500000208DF801000520FFF78FFF17E0052CEA
:103F600006DC01208DF801000520FFF786FF0EE03A
:103F7000142C06DC02208DF801000A20FFF77DFFDB
:103F800005E003208DF801001420FFF776FF9DF86F
:103F90000100072101EB8010C0B28DF80100404AFA
:103FA0001268917C3E4A526810786B460222FFF7F5
:103FB00003F810B14FF0FF30A4E7082138488172B0
:103FC00000210173012101750020FFF721FF00206E
:103FD00098E738B504463248807A10B94FF0FF3080
:103FE00038BD2F4890F8240010B14FF0FF30F7E7AC
:103FF0002B48007D50B134B1282C04DCE0B2FFF72F
:104000007BFF0020ECE70020FFF776FF042C01DAAD
:10401000042404E0B4F57A7F01DD4FF47A744FF4A0
:104020007A7090FBF4F0401EC0B200901C4A1268F7
:1040300051781B4A526810786B460122FEF7BCFF8C
:1040400010B14FF0FF30CBE79DF80000401C4FF45B
:104050007A7191FBF0F081B21148C1810146C989A2
:104060004810FFF70AFF0020BAE738B504460C48AD
:10407000807A10B94FF0FF3038BD022C06D0042CE6
:1040800007D0082C08D0102C0FD10BE00020009096
:104090000EE0082000900BE01020009008E00000E7
:1040A000D80000201820009002E04FF0FF30E3E736
:1040B00000BFF948407A9DF80010B0EBE10F01D144
:1040C0000020D9E7F44A1268D179F34A526810788F
:1040D0006B460122FEF770FF10B14FF0FF30CBE7C7
:1040E0009DF80000C110EC4841720020C4E738B5CB
:1040F0000446E948807A10B94FF0FF3038BDFA2CF9
:1041000009D0B4F5FA7F09D0B4F57A7F09D0B4F5B7
:10411000FA6F0CD108E0002000900BE0082000901E
:1041200008E01020009005E01820009002E04FF019
:10413000FF30E3E700BFD848007A9DF80010B0EBED
:10414000E10F01D10020D9E7D34A12689179D24A10
:10415000526810786B460122FEF72EFF10B14FF027
:10416000FF30CBE79DF80000C010CB49087200205B
:10417000C4E71CB580208DF80000C74A1268917C06
:10418000C54A526810786B460122FEF715FF10B140
:104190004FF0FF301CBD6420FDF772FF00208DF84A
:1041A0000000BD4A1268917CBB4A526810786B4689
:1041B0000122FEF701FF10B14FF0FF30EAE7B64AE7
:1041C0001268917DB44A526810786B460622FEF759
:1041D00057FF10B14FF0FF30DCE79DF80500C00736
:1041E000400F9DF8031001F0010140EA41009DF8E5
:1041F000011001F0010140EA010494B1012C03D146
:104200000121A548C17431E0022C03D10021A2484C
:10421000C1742BE02146A1A002F06CFB4FF0FF30EF
:10422000B8E79D4A1268D1789B4A526810786B466D
:104230000122FEF725FF10B14FF0FF30AAE79DF8ED
:10424000000000F00F042CB99E4802F053FB4FF021
:10425000FF309FE7042C06D19BA002F04BFB01210D
:104260008D48C17402E000218B48C174FF218A4847
:104270008172FF2088490872FF2187484172C1720C
:104280004FF6FF71C181FF21017481740121017317
:1042900080F82210002180F8231041750175163036
:1042A000016041608160163880F8241080F8251084
:1042B000C1844FF4FA60FFF71AFF10B14FF0FF30DE
:1042C00068E70220FFF7D1FE10B14FF0FF3061E741
:1042D0002A20FFF7D2FD10B14FF0FF305AE732200D
:1042E000FFF777FE10B14FF0FF3053E70020FFF7E4
:1042F0008FFD10B14FF0FF304CE70020FFF706FCB8
:1043000010B14FF0FF3045E70020FFF79AFB002087
:1043100040E770477CB504460D465F48807A00F060
:10432000700010B94FF0FF307CBD5B4A1268117B02
:10433000594A526810786B460622FEF7A1FE10B16A
:104340004FF0FF30F0E79DF801009DF8001040EAC3
:10435000012000B220809DF803009DF8021040EA81
:10436000012000B260809DF805009DF8041040EA2D
:10437000012000B2A08015B12846FFF7CAFF002037
:10438000D2E77CB504460D464348807A00F0080029
:1043900010B94FF0FF307CBD3F4A1268517B3E4A56
:1043A000526810786B460622FEF76AFE10B14FF095
:1043B000FF30F0E79DF801009DF8001040EA012071
:1043C00000B220809DF803009DF8021040EA012011
:1043D00000B260809DF805009DF8041040EA0120BD
:1043E00000B2A08015B12846FFF793FF0020D2E766
:1043F0002DE9FE4F05460C462748807A18B94FF044
:10440000FF30BDE8FE8F244A1268917B224A526831
:10441000107802AB0222FEF733FE10B14FF0FF30EE
:10442000EFE79DF809009DF8081040EA012006B268
:1044300014B12046FFF76DFF17494968C88804F09A
:10444000ABFC154901904968B1F9080004F08CFCF7
:104450008346304604F088FC5946009004F0ECFD99
:104460008246019904F04EFB81461F4904F0DCFAB4
:1044700080464FF08F4104F0D7FC074604F038FC2B
:1044800028600020BDE710B588B004461CB94FF085
:10449000FF3008B010BD29E0D8000020556E7375BC
:1044A00070706F7274656420736F66747761726583
:1044B0002070726F64756374207265762025642E97
:1044C0000A000000949F000848616C662073656EC6
:1044D0007369746976697479207061727420666F8B
:1044E000756E642E0D0A000000000C42206830B981
:1044F000606820B9A06810B9002008B010BDFA4962
:104500004968087806AB03221146FEF7B9FD10B1E1
:104510004FF0FF30F1E79DF81800082101EB201063
:1045200000F00F00ADF800009DF8190001EB20101D
:1045300000F00F00ADF802009DF81A0001EB20100A
:1045400000F00F00ADF8040020684100BDF9000044
:10455000403091FBF0F000B2ADF81000606841000F
:10456000BDF90200403091FBF0F000B2ADF812004E
:10457000A0684100BDF90400403091FBF0F000B2AA
:10458000ADF81400D8494968087806AB06221146F0
:10459000FEF776FD10B14FF0FF30AEE79DF8190041
:1045A0009DF8181040EA012000B2ADF808009DF80F
:1045B0001B009DF81A1040EA012000B2ADF80A0075
:1045C0009DF81D009DF81C1040EA012000B2ADF8D6
:1045D0000C00BDF81000BDF80810084400B2ADF89A
:1045E0001000BDF81200BDF80A10084400B2ADF882
:1045F0001200BDF81400BDF80C10084400B2ADF86C
:104600001400BDF81000000A8DF81800BDF8100065
:10461000C0B28DF81900BDF81200000A8DF81A001A
:10462000BDF81200C0B28DF81B00BDF81400000ADE
:104630008DF81C00BDF81400C0B28DF81D00AA4909
:104640004968087806AB06221146FEF7B5FC10B1A2
:104650004FF0FF3051E700204FE70146A248007AB3
:1046600030B1012807D0022809D003280FD10AE071
:10467000FA2008800EE04FF4FA7008800AE04FF448
:104680007A70088006E04FF4FA60088002E00020AB
:10469000088000BF00BF0020704701469248407A62
:1046A00030B1012807D0022808D003280CD108E037
:1046B000022008700BE00420087008E00820087051
:1046C00005E01020087002E04FF0FF30704700BF97
:1046D0008548C07C18B108784006000E087000209C
:1046E000F4E701468048C07A082817D2DFE800F0D6
:1046F0001704070A0D101318BC20088013E062206D
:10470000088010E02A2008800DE0142008800AE0CC
:104710000A20088007E00520088004E000BF00BFF1
:104720000020088000BF00BF0020704701466E488F
:1047300090F8240010B14FF0FF3070476A48C089EC
:1047400008800020F9E7014600200880401E7047DD
:1047500001464FF0FF30704701466348007A30B1A0
:10476000012807D0022808D003280CD108E05F48B0
:1047700008600BE05E48086008E05E48086005E0FD
:104780005D48086002E04FF0FF30704700BF002036
:10479000FBE701465448407A30B1012808D002288E
:1047A0000AD0032810D10BE04FF4804008800EE0BF
:1047B00041F69C7008800AE04FF48050088006E0C3
:1047C0004FF40060088002E04FF0FF30704700BFF8
:1047D0004548C07C10B10888401008800020F5E7EB
:1047E00001464148007C08700020704701463E4861
:1047F000807A10B10120087001E0002008700020CC
:10480000704738B504463848807A10B94FF0FF3009
:1048100038BD354A1268117C334A526810786B46AD
:104820000222FEF72DFC10B14FF0FF30F0E79DF8AB
:1048300001009DF8001040EA012000B22080002015
:10484000E6E72DE9FE4F0746884692461D46DDF80D
:1048500030B000260024244890F8240010B1601ED7
:10486000BDE8FE8F002028701F48807A10B94FF0F5
:10487000FF30F5E71C48007C10B94FF0FF30EFE740
:104880001948007C00F0400008B1B01CC6B21648C0
:10489000007C00F0200008B1B01CC6B21248007CB9
:1048A00000F0100008B1B01CC6B20F48007C00F048
:1048B000080008B1B01DC6B20B4A1268917A0A4AC4
:1048C000526810786B460222FEF7DAFB10B14FF007
:1048D000FF30C5E79DF801009DF8001040EA01296E
:1048E000B1450BDA0020BBE7D800002000000343ED
:1048F000000083423333034233338341FC48406832
:104900004088B9EB600F17DDF94A1268517CF84A0C
:10491000526810786B460122FEF7B2FB10B14FF0DF
:10492000FF309DE79DF8000000F0100020B1FFF778
:1049300091F96FF0010093E75046FFF7EAFCEC4A6B
:104940001268D17AEA4A526810786B463246FEF70E
:1049500097FB10B14FF0FF3082E799FBF6F0401E55
:104960008BF8000000202870B4422AD0E048007C78
:1049700000F0080028B3601C1DF800001DF80410AA
:1049800040EA012000B2A8F80000E01C1DF8001069
:10499000A01C1DF8000041EA002000B2A8F80200A7
:1049A000601D1DF80010201D1DF8000041EA0020C8
:1049B00000B2A8F80400287840F008002870A01D74
:1049C00084B2B44213D0CA48007C00F0400070B1F9
:1049D000601C1DF800001DF8041040EA012000B220
:1049E0003880287840F040002870A01C84B2B4427F
:1049F00013D0BF48007C00F0200070B1601C1DF88F
:104A000000001DF8041040EA012000B278802878E8
:104A100040F020002870A01C84B2B44213D0B448E7
:104A2000007C00F0100070B1601C1DF800001DF843
:104A3000041040EA012000B2B880287840F010004D
:104A40002870A01C84B200200AE7F8B504460F467F
:104A50001646A74890F8240010B94FF0FF30F8BD73
:104A6000A348807A10B94FF0FF30F8E7A04A1268E7
:104A7000917A9F4A526810786B460222FEF700FB3B
:104A800010B14FF0FF30EAE79DF801009DF80010EB
:104A900040EA0125A54203DA00203070401EDEE71F
:104AA000934840684088B5EB600F17DD904A126864
:104AB000517C8F4A526810786B460122FEF7E0FA6B
:104AC00010B14FF0FF30CAE79DF8000000F0100071
:104AD00020B1FFF7BFF86FF00100C0E7E2B2844BEE
:104AE0001B68D97A824B5B6818783B46FEF7C8FA98
:104AF00010B14FF0FF30B2E795FBF4F0401E30707C
:104B00000020ACE701467A4880F822100020704768
:104B10007CB5054676494968087801AB04220D2129
:104B2000FEF7AEFA08B107207CBD9DF80700C0F380
:104B300001109DF8041001F0E00140EAE1008DF859
:104B400000009DF80700C0F381009DF8051001F0FA
:104B5000E00140EAE1008DF801009DF8070000F057
:104B600003009DF8061001F0E00140EAE1008DF835
:104B7000020000241CE01DF8040018B9002045F8CC
:104B8000240013E05B4845F8240006E055F82400B3
:104B9000594904F049F945F824001DF80400401E65
:104BA000C0B20DF804000028F0D100BF601CC4B2F0
:104BB000032CE0DB0020B7E72DE9FE4F06460F4649
:104BC00000256846FFF7A4FF002442E056F82400C1
:104BD00057F82410A0EB010ABAF1000F01DB51468F
:104BE00001E0CAF10001084604F0BEF883464FF028
:104BF0008F4103F087FF80465DF82400002104F018
:104C000043F816D05DF82410404603F07BFF82463F
:104C10004FF07E5104F010FA814629F0004A3748DF
:104C2000416A504604F0CCF912D20120A04005435D
:104C30000EE03248C169404604F0C2F805D32F485F
:104C4000016A404604F0BCF902D20120A0400543AD
:104C5000641C032CBADB2846BDE8FE8F2DE9FC5FFF
:104C600006460F46002522494968087801AB032211
:104C70000D21FEF705FA10B10720BDE8FC9F9DF855
:104C8000040000F01F008DF804009DF8050000F0FE
:104C90001F008DF805009DF8060000F01F008DF83C
:104CA0000600002462E056F8240057F82410A0EB18
:104CB000010BBBF1000F01DB594601E0CBF1000114
:104CC000084604F051F84FF08F41009003F01AFFAE
:104CD000814601A8005DC0B30849086804F05CF88B
:104CE00083465946064803F00DFF80460FE000005A
:104CF000D80000207B14AE3E1D5A843F409200082D
:104D000000B04C45FE49404604F08EF8804601A8AC
:104D1000005D401EC0B201A908550028F2D14146ED
:104D2000484603F0EFFE83464FF07E5104F084F9CD
:104D300082462AF0004BF3488169584604F040F956
:104D400013D20120A04005430FE0FFE7ED480169C1
:104D5000484604F035F805D3EA484169484604F06E
:104D60002FF902D20120A0400543641C032C9ADBDA
:104D7000284682E72DE9F04F87B005460C4691465C
:104D800001208DF8100000208DF81100DE4A126815
:104D9000917CDD4A5268107804AB0222FEF70CF9D0
:104DA00020B14FF0FF3007B0BDE8F08FC820FDF70D
:104DB00067F900208DF81000D34A1268D17BD24ADF
:104DC0005268107804AB0122FEF7F6F810B14FF0EC
:104DD000FF30E8E7CC4A12685179CB4A5268107824
:104DE00004AB0122FEF7E8F810B14FF0FF30DAE72C
:104DF000C54A1268917CC44A5268107804AB0122FB
:104E0000FEF7DAF810B14FF0FF30CCE7BE4A126877
:104E1000D17DBD4A5268107804AB0122FEF7CCF870
:104E200010B14FF0FF30BEE7B74A12681179B64AA9
:104E30005268107804AB0122FEF7BEF810B14FF0B3
:104E4000FF30B0E70C208DF81000AF4A12681179DE
:104E5000AD4A5268107804AB0122FEF7ADF810B1EC
:104E60004FF0FF309FE70F20FDF70AF9A648806A50
:104E7000407A8DF81000A44A12689178A24A5268CC
:104E8000107804AB0122FEF797F810B14FF0FF3015
:104E900089E79D48806A007A8DF810009A4A126866
:104EA0005178994A5268107804AB0122FEF784F8D1
:104EB00010B14FF0FF3076E7B9F1000F07D09248FC
:104EC000806A807A40F0E0008DF8100004E08E489F
:104ED000806A807A8DF810008B4A126891798A4A2C
:104EE0005268107804AB0122FEF766F810B14FF05B
:104EF000FF3058E7B9F1000F07D08348806AC07AC5
:104F000040F0E0008DF8100003E07E48C07A8DF894
:104F100010007D4A1268D1797B4A5268107804AB40
:104F20000122FEF749F810B14FF0FF303BE7B9F12D
:104F3000000F02D0C820FDF7A3F840208DF8100024
:104F4000714A12681179704A5268107804AB0122D4
:104F5000FEF732F810B14FF0FF3024E778208DF8DB
:104F60001000694A12685179674A5268107804AB98
:104F70000122FEF721F810B14FF0FF3013E761492D
:104F80008889FDF77DF800208DF810005E4A1268D0
:104F900051795D4A5268107804AB0122FEF70CF893
:104FA00010B14FF0FF30FEE6574A1268917A564A28
:104FB0005268107804AB0222FEF762F810B14FF08D
:104FC000FF30F0E69DF811009DF8101040EA012B2B
:104FD0000C209BFBF0F0C6B20020A860686028603F
:104FE000A06060602060824665E0474A1268D17A1E
:104FF000454A5268107804AB0C22FEF741F810B114
:105000004FF0FF30CFE69DF811009DF8101040EAF8
:10501000012000B2ADF808009DF813009DF81210B1
:1050200040EA012000B2ADF80A009DF815009DF895
:10503000141040EA012000B2ADF80C00BDF90810D0
:10504000206808442060BDF90A1060680844606068
:10505000BDF90C10A0680844A0609DF817009DF8E9
:10506000161040EA012000B2ADF800009DF81900CA
:105070009DF8181040EA012000B2ADF802009DF83A
:105080001B009DF81A1040EA012000B2ADF80400A0
:10509000BDF90010286808442860BDF9021068684E
:1050A00008446860BDF90410A8680844A8600AF1C3
:1050B000010000F0FF0AB24597DB1248D0F800C0AB
:1050C0002868C117090441EA104107046246002319
:1050D000384601F0EAFB32460023CDE9020101F037
:1050E000E4FB28600748D0F800C06868C1170904CD
:1050F00041EA1041070462460023384606E00000FA
:1051000054E3853F40920008D800002001F0CDFB19
:1051100032460023CDE9020101F0C7FB6860FE487A
:10512000D0F800C0A868C117090441EA104107047B
:1051300062460023384601F0B8FB32460023CDE931
:10514000020101F0B2FBA860F348D0F804C0216866
:10515000C817000440EA11480F046246002338468D
:10516000414601F0A2FB32460023CDE9020101F0E5
:105170009CFB2060E848D0F804C06068C1170904AF
:1051800041EA1041070462460023384601F08DFBD6
:1051900032460023CDE9020101F087FB6060DE4862
:1051A000D0F804C0A068C117090441EA10410704FF
:1051B00062460023384601F078FB32460023CDE9F1
:1051C000020101F072FBA060A068002804DDA06865
:1051D000A0F58030A06003E0A06800F58030A060FA
:1051E0000020E0E538B50446CC4890F82400A04201
:1051F00001D1002038BD24B3C84890F8250010B96B
:105200004FF0FF30F6E70020FEF75EFB0020FEF7D0
:105210007DFCC249C88CFEF7DCFE00200090BF492F
:10522000496808786B4601222321FDF7C5FE01215C
:10523000BA4880F824100120FEF746FBFEF70AFD6D
:1052400013E00020FEF740FBB448007C0090B34917
:10525000496808786B4601222321FDF7ADFE002145
:10526000AE4880F82410FEF7F5FC0020C2E72DE9D7
:10527000F04F8DB083460F4602200C90A74890F85F
:10528000240020B10020FFF7ADFF012600E000263A
:1052900003A8FFF7E2F905A8FFF7FFF901A8FFF758
:1052A00020FA02A8FFF742FA9C4890F80AA004A846
:1052B000FFF796FA002407E0002239465846FFF728
:1052C00059FD00B902E0641C022CF5DB00BF022C82
:1052D00001D1002528E0002407E0012206A909A841
:1052E000FFF748FD00B902E0641C022CF5DB00BFAB
:1052F000022C01D1002517E006A93846FFF75CFC17
:1053000000F0FF0809A95846FFF7A8FC00F0FF09C4
:105310000025B9F1000F01D145F00105B8F1000FEA
:1053200001D145F0020500BFFF207C490872FF2132
:105330007A484172C1724FF6FF71C181FF218172BB
:10534000017401210173BDF80C00FEF7D0FE9DF839
:105350001400FEF78AFEBDF80400FEF78EFDBDF8CE
:105360000800FEF736FE5046FEF76BFB9DF8100076
:10537000FEF74EFD16B10120FFF734FF28460DB0B1
:10538000BDE8F08FF8B504460D46164616B94FF045
:10539000FF30F8BD6148807A10B94FF0FF30F8E770
:1053A00020128DF80000E0B28DF801009DF8010098
:1053B00028445A4949684989884202DD4FF0FF3044
:1053C000E7E7564A1268117E544A526810786B46D5
:1053D0000222FDF7F1FD10B14FF0FF30D9E7EAB23C
:1053E0004E4B1B68597D4D4B5B6818783346FDF773
:1053F000E3FD10B14FF0FF30CBE70020C9E7F8B56F
:1054000004460D46164616B94FF0FF30F8BD434826
:10541000807A10B94FF0FF30F8E720128DF80000C5
:10542000E0B28DF801009DF8010028443B4949682D
:105430004989884202DD4FF0FF30E7E7374A1268BA
:10544000117E364A526810786B460222FDF7B4FD91
:1054500010B14FF0FF30D9E7EAB2304B1B68597DED
:105460002E4B5B6818783346FDF70AFE10B14FF0FB
:10547000FF30CBE70020C9E72DE9F04385B00546B2
:105480000E4690469946254890F8250020B14FF0E9
:10549000FF3005B0BDE8F08316B94FF0FF30F8E7F4
:1054A000002423E0281B102801DD102000E0281B29
:1054B00087B2321939462046FFF764FF10B14FF02A
:1054C000FF30E6E701AA39462046FFF798FF10B102
:1054D0004FF0FF30DDE730193A4601A901F015FB26
:1054E00010B16FF00100D4E7E01984B2AC42D9DB0F
:1054F0004FEA28208DF8000008F0FF008DF8010029
:10550000064A1268917E054A526810786B4602225C
:10551000FDF752FD38B103E040920008D8000020AA
:105520004FF0FF30B5E701218A4880F82510A0F838
:1055300026900020ADE70146864890F824000870C8
:105540000020704702464FF0FF30704701464FF091
:10555000FF307047F8B505460F461446002C70D052
:10556000B5F5FF5F01DDFF2605E0202D01DA0126FC
:1055700001E0C5F3471607B90127282C02DD4FF0DB
:10558000FF30F8BD7348407D28BB724890F8240076
:1055900038B10020FFF726FE01216E4880F8201068
:1055A00003E000216B4880F820106A481630FFF7AE
:1055B00054F868481830FFF770F866481A30FFF75B
:1055C00090F864481C30FFF7B1F86248817A81771F
:1055D0001F30FFF705F90020FEF776F90020FEF7EF
:1055E0008BFC00208DF800005A4A12689178594AC5
:1055F000526810786B460122FDF7DEFC10B14FF0C7
:10560000FF30BEE740208DF80000524A1268D17B7F
:10561000504A526810786B460122FDF7CDFC00B16C
:1056200065E08DF800608DF801704A4A1268117AC1
:10563000484A526810786B460222FDF7BDFC08B15B
:1056400055E047E00520FCF71BFD4248407A072162
:1056500001EBC000C0B28DF800003E4A1268D1795B
:105660003C4A526810786B460122FDF7A5FC00B158
:105670003DE020208DF80000012C03D100208DF8A2
:1056800001000EE0052C03DC01208DF8010008E08C
:10569000142C03DC02208DF8010002E003208DF8B9
:1056A00001009DF80100072101EB8010C0B28DF8C8
:1056B0000100284A1268917C264A526810786B468D
:1056C0000222FDF779FC00B111E00121214841756A
:1056D000002056E71F4A1632002103E0505C00B15B
:1056E00005E0491C0C29F9D34FF0FF3049E7FF20B2
:1056F00018490872FF2117484172C1724FF6FF71B5
:10570000C181FF2181720174012101730146887FEB
:10571000FEF797F90F49C88AFEF7E9FC0D49087EA4
:10572000FEF7A3FC0B49488BFEF7A7FB0949888BC2
:10573000FEF74FFC0749C87FFEF76AFB054890F863
:10574000200010B10120FFF74DFD002101484175F7
:10575000002016E7D800002010B5C8234FF480625F
:10576000F74940F6F630FFF787FE10BD10B586B05A
:105770000446F4A000680390F3A000680290F3A030
:1057800000680190F2A00068009004F0030003A9F3
:10579000085C8DF8140003A8C4F3C101405C8DF8C7
:1057A000150003A8C4F38111405C8DF8160004F0C5
:1057B000030002A9085C8DF8100002A8C4F3C1011F
:1057C000405C8DF8110002A8C4F38111405C8DF893
:1057D000120005AA032140F22640FFF7D3FD18B1BD
:1057E0004FF0FF3006B010BD04AA032140F22A405A
:1057F000FFF7C8FD10B14FF0FF30F3E701980590B7
:105800000098049004F0040058B19DF8140040F092
:1058100001008DF814009DF8100040F001008DF893
:10582000100004F0200058B19DF8150040F0010070
:105830008DF815009DF8110040F001008DF8110061
:1058400004F4807058B19DF8160040F001008DF806
:1058500016009DF8120040F001008DF8120005AA14
:1058600003214FF48860FFF78DFD10B14FF0FF303A
:10587000B8E704AA032140F23140FFF783FD10B1DD
:105880004FF0FF30AEE7B34804810020AAE71FB510
:105890000446B048007A00F0030054F8200001905C
:1058A000AC48007A00F0040010B101984042019029
:1058B000A848007AC0F3C10054F820000290A5481F
:1058C000007A00F0200010B1029840420290A148F6
:1058D000007AC0F3811054F8200003909D4800899D
:1058E00000F4807010B10398404203909A490198E7
:1058F00080FB0101800F40EA8100019096490298E7
:1059000080FB0110820042EA917002909249039854
:1059100080FB0110820042EA917003900198000E12
:105920008DF800000198000C8DF801000198000A24
:105930008DF802000198C0B28DF803006A46042178
:105940004FF47470FFF71EFD18B14FF0FF3004B034
:1059500010BD0298000E8DF800000298000C8DF822
:1059600001000298000A8DF802000298C0B28DF87A
:1059700003006A4604214FF47570FFF703FD10B170
:105980004FF0FF30E3E70398000E8DF80000039816
:10599000000C8DF801000398000A8DF802000398AE
:1059A000C0B28DF803006A4604214FF47670FFF709
:1059B000E9FCCCE770B588B0064601A8FEF7E9FE21
:1059C000BDF804000021C90341EA5045C403614801
:1059D000007A00F0030056F8200005905D48007A38
:1059E00000F0040010B10598404205905948007A33
:1059F000C0F3C10056F8200006905648007A00F027
:105A0000200010B10698404206905248007AC0F338
:105A1000811056F8200007904E48008900F48070ED
:105A200010B10798404207900598C117A0FB0423C6
:105A300001FB043100FB0510810041EA92700590E2
:105A40000698C117A0FB042301FB043100FB0510DD
:105A5000810041EA927006900798C117A0FB0423C9
:105A600001FB043100FB0510810041EA92700790B0
:105A70000598000E8DF808000598000C8DF80900B7
:105A80000598000A8DF80A000598C0B28DF80B0041
:105A90000698000E8DF80C000698000C8DF80D008D
:105AA0000698000A8DF80E000698C0B28DF80F0017
:105AB0000798000E8DF810000798000C8DF8110063
:105AC0000798000A8DF812000798C0B28DF81300ED
:105AD00002AA0C214FF42570FFF754FC08B070BDEA
:105AE00030B585B004461DA207CA02AB07C3C82C57
:105AF00003DD4FF0FF3005B030BDC82090FBF4F05F
:105B0000401E85B2280A8DF80000E8B28DF8010029
:105B10006A46022140F21620FFF734FC10B14FF024
:105B2000FF30E8E702AA0C2140F6C120FFF72AFC6B
:105B300010B14FF0FF30DEE7064884810020DAE73D
:105B4000689200084CCD6C000CC92C0036567600CB
:105B500026466600B401002009E3CA02FEF2ABC487
:105B6000AAF1DFDFBBAFDFDF0146FC488089088098
:105B7000002070472DE9FC4706460F4606F0070057
:105B800010B1B7F5C86F03DD4FF0FF30BDE8FC87FB
:105B9000384603F001F98146F14902F0B3FF80462F
:105BA0006846FEF77AFD9DF80000022806D004281A
:105BB00016D0082826D0102848D135E04FF08D4166
:105BC000404603F031F9814603F0AEF884B2E5496E
:105BD000404603F029F9814603F0A6F885B238E083
:105BE0004FF08C41404603F01FF9814603F09CF8CA
:105BF00084B2DD49404603F017F9814603F094F87A
:105C000085B226E04FF08B41404603F00DF9814606
:105C100003F08AF884B2D549404603F005F981467D
:105C200003F082F885B214E04FF08A41404603F059
:105C3000FBF8814603F078F884B2CD49404603F082
:105C4000F3F8814603F070F885B202E04FF0FF30C0
:105C50009CE700BF20128DF80400E0B28DF805002B
:105C600028128DF80600E8B28DF8070006F0010052
:105C7000A0B101AA02214FF4EA70FFF783FB10B133
:105C80004FF0FF3082E70DF1060202214FF49270CF
:105C9000FFF778FB10B14FF0FF3077E706F0020016
:105CA000A0B101AA02214FF4EC70FFF76BFB10B119
:105CB0004FF0FF306AE70DF1060202214FF49470B5
:105CC000FFF760FB10B14FF0FF305FE706F0040014
:105CD000A0B101AA02214FF4EE70FFF753FB10B1FF
:105CE0004FF0FF3052E70DF1060202214FF496709B
:105CF000FFF748FB10B14FF0FF3047E7002045E7C2
:105D000038B504460020009004F0010020B19DF851
:105D1000000040F03000009004F0020020B19DF837
:105D2000000040F00C00009004F0040020B19DF849
:105D3000000040F0030000906A4601214FF4A47077
:105D4000FFF720FB38BD38B50446012C01DA0124E9
:105D500002E0042C00DD0424601EC0B200906A46FC
:105D6000012140F24F10FFF70DFB38BD38B5044656
:105D7000052094FBF0F085B228128DF80000E8B2FF
:105D80008DF801006A4602214FF4EF70FFF7FAFA2E
:105D900038BD38B50446052094FBF0F085B22812D2
:105DA0008DF80000E8B28DF801006A4602214FF438
:105DB000ED70FFF7E7FA38BDF8B505460E464FF42B
:105DC0007A7095FBF0F000FB06F4200E8DF80000D1
:105DD000200C8DF80100200A8DF80200E0B28DF849
:105DE00003006A4604214FF4AE70FFF7CBFAF8BD0A
:105DF00038B50446052094FBF0F084B220128DF8EB
:105E00000000E0B28DF801006A4602214FF4AD7047
:105E1000FFF7B8FA38BD38B50446052094FBF0F01A
:105E200084B220128DF80000E0B28DF801006A46BD
:105E300002214FF4AC70FFF7A5FA38BD38B504461F
:105E400014B94FF0FF3038BD6A4604214FF4587042
:105E5000FFF7D5FA10B14FF0FF30F4E79DF80000DE
:105E600000069DF8011040EA01409DF8021040EA4A
:105E700001209DF80310084320600020E3E738B5B7
:105E80000446200E8DF80000200C8DF80100200A39
:105E90008DF80200E0B28DF803006A4604214FF449
:105EA0005870FFF76FFA38BD38B5044614B94FF093
:105EB000FF3038BD6A4604214FF47170FFF79FFA36
:105EC00010B14FF0FF30F4E79DF8000000069DF898
:105ED000011040EA01409DF8021040EA01209DF8BF
:105EE0000310084300EB8000800020600020E0E702
:105EF00038B504461420B4FBF0F4200E8DF80000F1
:105F0000200C8DF80100200A8DF80200E0B28DF817
:105F100003006A4604214FF47170FFF733FA38BD6D
:105F200038B5044664B120208DF8000028208DF893
:105F3000010030208DF8020038208DF8030004E0C5
:105F4000A3220421684600F00CFE6A46042140F6B4
:105F50009E20FFF717FAFDF77DFE38BDB401002043
:105F600000004843000040460000C0450000404596
:105F70000000C04438B5044664B1C0208DF800006C
:105F8000C2208DF80100C4208DF80200C6208DF8D3
:105F9000030004E08B220421684600F0E2FD6A461B
:105FA000042140F69820FFF7EDF9FDF753FE38BDC8
:105FB0003EB504466CB1FDA1D1E900208968CDE968
:105FC000002002916A4609214FF49760FFF7DAF941
:105FD0003EBDF9A2D2E900109268CDE9010200911C
:105FE0006A4609214FF49760FFF7CCF9F0E73EB518
:105FF000044602208DF80000CA208DF80100E3203D
:106000008DF8020009208DF803006A4604216820FB
:10601000FFF7B8F9A3208DF8000004F0400048B164
:10602000C0208DF80100C8208DF80200C2208DF834
:10603000030006E0A3208DF801008DF802008DF822
:10604000030004F4C07048B1C4208DF80400CC20D3
:106050008DF80500C6208DF8060006E0A3208DF817
:1060600004008DF805008DF80600A3208DF80700C8
:106070008DF808008DF809006A460A2140F6A7202D
:10608000FFF780F904F0030018B120208DF800001C
:1060900002E0D8208DF800006A46012140F6B620C3
:1060A000FFF770F904F0200018B10120FFF780FF1E
:1060B00002E00020FFF77CFF04F4C07008B304F492
:1060C000807060B1B2208DF800008B208DF8010047
:1060D000B6208DF802009B208DF803000BE0B02065
:1060E0008DF8000080208DF80100B4208DF80200AA
:1060F00090208DF803006A46042140F6A220FFF7A5
:1061000041F904F0010020B3F8208DF800006A4640
:1061100001214FF40B60FFF735F9FA210720FFF753
:1061200029FD0720FFF7ECFD0120FFF70CFE64209E
:10613000FFF71CFE4FF4FA70FFF72BFEC821A148B1
:10614000FFF73AFE2820FFF753FE0A20FFF763FE11
:1061500008E0D8208DF800006A4601214FF40B605A
:10616000FFF710F904F0020018B1D9208DF80000F3
:1061700002E0D8208DF800006A46012140F23D700F
:10618000FFF700F904F0040018B10120FFF7F2FE58
:1061900002E00020FFF7EEFE04F0100018B101202D
:1061A000FFF7BEFE02E00020FFF7BAFE44F0080051
:1061B00085494881FDF74EFD00208349887304F02E
:1061C000400018B10846807B801D887304F4C070BD
:1061D00020B17D48807B801D7B49887304F01400CA
:1061E00020B17948807B10307749887304F0030030
:1061F00020B17548807B001D7349887300203EBD27
:106200000146714840890880002070472DE9F0411F
:106210000446E07800F0C006E07800F03F056078C2
:1062200000F0010098B1EF102846E91705EB517115
:10623000C910A5EBC101491C01F0FF0862480068C4
:1062400020B16148414602683846904700BF6078F7
:1062500000F0080030B15C48406818B1B0115A4AEB
:10626000516888470020BDE8F08110B586B004462B
:1062700056A207CA03AB07C357A207CA8DE8070097
:10628000012C09D0022C0ED103AA0B2140F682204A
:10629000FFF778F806B010BD6A460B2140F6822061
:1062A000FFF770F8F6E74FF0FF30F3E72DE9F04F16
:1062B0008DB00746884615469946DDE9166B0024E1
:1062C000002030804049887B5A4605A9FEF7BDFB77
:1062D00018B1601E0DB0BDE8F08F3B48807A00F029
:1062E0001400002861D09DF8140000069DF81510D8
:1062F00040EA01409DF8161040EA01209DF8171071
:10630000084328609DF8180000069DF8191040EA1F
:1063100001409DF81A1040EA01209DF81B10084327
:1063200068609DF81C0000069DF81D1040EA0140C1
:106330009DF81E1040EA01209DF81F100843A86038
:106340009DF8200000069DF8211040EA01409DF8CC
:10635000221040EA01209DF823100843E86004F170
:106360001000C4B2286800140190686800140290FC
:10637000A86800140390E868001404900198404352
:10638000029901FB0100039901FB0100049901FB43
:10639000010ABAF1706F02DBBAF1885F22DDFDF706
:1063A00059FC00203080401E94E721E0B8AAB38D4C
:1063B000B4980D355D000000B8AAAAAAB088C3C57C
:1063C000C700000009E3CA02B4010020D8B1B9F344
:1063D0008BA391B609B4D900DAB1B9F38BA391B606
:1063E000DAB4DA00B6F9000040F48070308000BF03
:1063F0003448807A00F0400020B305A9601C085C96
:10640000095D40EA012000B2A8F8000005A9E01CDF
:10641000095C05AAA01C105C41EA002000B2A8F8A3
:10642000020005A9601D095C201D105C41EA0020E6
:1064300000B2A8F80400A01DC4B2B6F9000040F0F4
:10644000080030801F48408900F4C07008B305A9D7
:10645000601C085C095D40EA012000B2388005A993
:10646000E01C095C05AAA01C105C41EA002000B2F7
:10647000788005A9601D095C201D105C41EA0020A0
:1064800000B2B880A01DC4B2B6F9000040F07000A0
:1064900030800C48807A00F0030018B105A9081973
:1064A000FFF7B4FE4846FDF734FF002012E701462F
:1064B0000448016000207047014602484160002006
:1064C00070470000B4010020704770B505468D4943
:1064D000284602F075FC08D38B49284602F070FD6F
:1064E00003D38A480078012801D1012400E0002468
:1064F000204670BD03461846884200DD084690429B
:1065000000DA104670472DE9FF5F0446894680484F
:1065100003908048029004EB0901484202F024FCF9
:106520007D4908607D48006802F052FA07467C4ABF
:106530007C4B02F059F8054601F004FE77490860EB
:106540007548006802F044FA754A774BCDE90001BE
:1065500002F04AF805460E467048006802F038FA24
:1065600007462A46334601F01FFE824601F0EAFD47
:106570006A490860084601686C48006802F054FAED
:106580006A4908606A496948006802F019FD02D248
:1065900067486649086067496448006802F010FC73
:1065A00002D264486149086060480299006802F0BC
:1065B0003BFC07465948006880F000463046039986
:1065C00002F032FC0546394602F036FD5A490860B1
:1065D0005A480068FFF779FF012803D04B4800783C
:1065E000012802D10020514908605348006802F098
:1065F0007FFB04B0BDE8F09F2DE9FE4F04460D4639
:106600004F4E504F0021204602F00BFD02902946CC
:10661000002002F011FD01903946019802F004FCBF
:1066200086F0004B00905846029902F0FDFB82462E
:10663000009902F001FD814602F05AFB8046404677
:10664000BDE8FE8F10B5FDF75BF83F4800683B4999
:1066500008603E49B1F9000002F086FB3C49086041
:1066600010BD2DE9F0414FF480503A4908603A4896
:10667000007808B9012000E0002037490870FFF7D2
:10668000E1FF35480078012802D10020BDE8F08103
:106690002F48016829480068FFF7AEFF04462F48DD
:1066A00001682F480068FFF72EFF05466719661935
:1066B0002C4A51423846FFF71DFF0746294A5142EE
:1066C0003046FFF717FF06461C480068FFF7FDFE3F
:1066D00018B931463846FFF7F7FE0020D6E7012803
:1066E00007D10A49097809B9012100E00021074AC8
:1066F000117070470146002901DA484200E008465F
:1067000070470000000020C2000020420C01002061
:1067100000002043CDCC4C3F140100201801002084
:106720009A9999999999E93F9999C93F1C01002033
:1067300000401C4600401CC610010020040100203F
:1067400000006143713D8A3FB4000020A00000209A
:1067500008010020140401400D0100206000002009
:106760005C0000200CE5FFFFFBF750FB4FF41650D8
:10677000FCF700F939A13E48FCF7C6F9FCF706FB27
:10678000FBF79DFD3BA13A48FCF7BEF9FCF76AFF19
:10679000FCF782FF60E00A20FBF772FC06213B4811
:1067A000FCF746FA3948C078B12806D13748007955
:1067B000B52802D100203549C8703448C078B328C4
:1067C00006D132480079B72802D100202F49C8707D
:1067D0002E48C078B22805D12C480079B62801D1BE
:1067E000FCF7B4FA2948C078B4280ED127480079BC
:1067F000B8280AD1FCF7BAFA4FF4FA70FBF740FC5C
:10680000FCF7A4FA00202149C8702048C078B528B8
:1068100005D11E480079B92801D1FCF7B7FA1B4809
:10682000C078B6280ED119480079BA280AD1FCF7E9
:10683000A5FA4FF4FA70FBF723FCFCF787FA002067
:106840001249C8701148C078B82805D10F4800799E
:10685000BC2801D1FCF782FA9DE70000496E6974FB
:1068600020426C756520746F6F74682E2E0D0A00BF
:10687000004400404D5055363035305F696E6974C4
:1068800069616C697A652E2E0D0A0000C401002032
:10689000704700BFFEE700BFFEE700BFFEE700BF96
:1068A000FEE7704770477047704710B54C1084EA98
:1068B000530404D54042C1F1000138BF491E1B42B8
:1068C00004D55242C3F1000338BF5B1E00F055F9F6
:1068D00014F0804F04D04042C1F1000138BF491E7E
:1068E00014F0004F04D05242C3F1000338BF5B1EC6
:1068F00010BD00000FB4044910B503AA029800F0BF
:1069000037FC10BC5DF814FB380000200FB41CB538
:10691000074B06AA7B4469460090059800F00FFCDF
:106920000020694600F01EFC1CBC5DF814FB000052
:106930004D08000070B5044685690068C10601D5A0
:10694000302600E02026C00707D070BDD4E9012121
:1069500030469047206A401C20626D1EF6D570BDFF
:1069600070B5044685690078C00707D170BDD4E9C9
:10697000012120209047206A401C20626D1EF6D520
:1069800070BD00002DE9F04106460024106875290D
:10699000314616A510D0AFF30080002802DA40423D
:1069A00013A507E031688A0701D512A502E049075F
:1069B00004D511A5012401E0AFF3008000210A22D3
:1069C00006F1240709E0B0FBF2FCB0FBF2F302FB96
:1069D0001C00303078541846491C0028F3D1234657
:1069E0002A463046BDE8F04100F03EB90000000004
:1069F0002D0000002B000000200000002DE9F047D2
:106A00004FF0000A89460446C0F820A02046E168FD
:106A10008847002876D0252806D0D4E90121904760
:106A2000206A401C2062F1E7E16820460025884783
:106A3000C4F81CA006460027C4F818A02A2E09D0C6
:106A4000304601F091F938B304EB8708303EC8F8BE
:106A5000186019E059F8041B204604EB8702916185
:106A6000E1688847012F064618D1E069002820DA3E
:106A700025F020051DE0D8F8180000EB800006EB9B
:106A800040003038C8F818002046E16888470646BC
:106A900001F06AF90028EED1012F0AD02E2E08D17C
:106AA0002046E16888477F1C0646022F45F02005F6
:106AB000C4DBA069002803DA404245F00105A0616B
:106AC000E80701D025F01005B6B1A6F1410019285C
:106AD00002D8203645F400654A46314620462560F6
:106AE0004D46F9F75FFB58B1012806D0ED1D25F0A2
:106AF000070000F1080989E704E005F1040985E7CA
:106B000030468AE7206ABDE8F08740EA010310B505
:106B10009B070FD1042A0DD310C808C9121F9C422D
:106B2000F8D020BA19BA884201D9012010BD4FF01F
:106B3000FF3010BD1AB1D30703D0521C07E000206C
:106B400010BD10F8013B11F8014B1B1B07D110F8C9
:106B5000013B11F8014B1B1B01D1921EF1D11846CC
:106B600010BD02F0FF0343EA032242EA024200F0B2
:106B700013BB704770477047704753EA020C00F030
:106B800069802DE9F04B4FF00006002B1FBFB3FAD0
:106B900083F503FA05F424FA05F65E4012BF1643A6
:106BA000B2FA82F502FA05F4C5F120051EBF22FAF9
:106BB00005FC44EA0C04203556EA044C4FEA144420
:106BC00018BF641C4FF000084FF00009904271EBB1
:106BD000030C39D3002919BFB1FA81F701FA07F67E
:106BE000B0FA80F700FA07F6C7F120071EBF20FAB7
:106BF00007FC46EA0C062037B6FBF4FCA7EB0507BA
:106C0000103F07F01F0BCBF120060CFA0BFB2CFA00
:106C100006F644BFB3460026202FA4BF5E464FF0C1
:106C2000000B5BEA060C08BF4FF0010B19EB0B09D8
:106C3000ABFB027C48EB0608C01B06FB02CC0BFB3F
:106C400003CC71EB0C01C1E70B46024641464846B6
:106C5000BDE8F08B13B54FF000004FF00001AFF32B
:106C60000080BDE81C4070472DE9F0470D4699466D
:106C70009246044600F124080168880604D5E069BC
:106C800021F01001216000E00120A84201DD471B36
:106C900000E00027A1697A1902EB0900081AA06137
:106CA0002078C00602D42046FFF744FE002608E004
:106CB000D4E901211AF806009047206A401C761C8E
:106CC00020624E45F4DB2078C0060AD52046FFF747
:106CD00031FE06E0D4E9012130209047206A401CB3
:106CE0002062381EA7F10107F4DC07E0D4E9012196
:106CF00018F805009047206A401C2062281EA5F164
:106D00000105F3DC2046FFF72BFE2078000602D5B4
:106D10000220BDE8F0870120FBE770472DE9FF4F17
:106D20000C461E464FF0FF378BB0D2E90001DDF86C
:106D300060800A908A46C1F30A5505B93D46002194
:106D400008464FF00000BAF1000F00F4400005DAE9
:106D500000EB80004FF4400101EA50004FEA9059E7
:106D6000B9F1010F00DDB9460A9850EA4A000ED089
:106D700044F61050A5F2FF3545432F14B8F1000F2B
:106D80001ED07542291E1EDDC9F100021CE0B8F1BB
:106D9000010F4FF0000001D0302103E0F24305E085
:106DA0002154401CB042FBDB30460022002121541C
:106DB0000B99C1F80880C1E900200FB0BDE8F08F41
:106DC000BD1B6D1CDEE74A4600DA694206A800F0EA
:106DD0008DFA06AB93E8070003AB83E80700504643
:106DE0000A9900F08FFB8DE80700A0F500501F38CE
:106DF00000900398002D09DD42F21F014A46084425
:106E000003A90390684600F0EEFD08E0A0F50050ED
:106E10004A461F3803A90390684600F0F8FD8DE844
:106E200007000004000C03D04FF0FF30410800E0E1
:106E30001046B8F1000F03D00022009215461EE064
:106E4000751E05D400F0CCF9303262556D1EF9D5AF
:106E5000B3460122084302D000227F1C04E02078C0
:106E6000302801D100227F1E002A099786D01DE01C
:106E7000112D07DA00F0B4F9303262556D1C50EA7A
:106E80000102F5D1084302D00098C8B10EE00021FC
:106E9000681E05E0235C625C63542254401E491C5A
:106EA0008142F7DBAB46A81B401E0990002004F886
:106EB0000B000B98099AC0F80880C0E9002B7CE70A
:106EC00011264FF0000859E72DE9F04F8846044697
:106ED000D21D22F0070191B0D1E90001CDE90A01EC
:106EE00000F0CBFE02460B98C00F01D02D2007E02A
:106EF0002068810701D52B2002E0202101EAC00093
:106F0000032A099001D0072A05DB034641462046A3
:106F100000F0ACF90BE12078800601D5E06900E0D3
:106F20000620B8F1650F814606D0B8F1660F18D07B
:106F3000B8F1670F70D131E00020B9F1110F009066
:106F400001DB112301E009F101030AAA01A90CA840
:106F5000FFF7E4FEDDE90C70002609F10105834628
:106F600047E001204B4600904FF000470AAA01A9D4
:106F70000CA8FFF7D3FEDDE90DB00C995D460026A5
:106F800010B909F101000D18B9EB050003D4C0F1E7
:106F9000FF3609F10105A5EB09002BE0B9F1010F5E
:106FA00001DA4FF001090020B9F1110F00904846B5
:106FB00001DD112300E003460AAA01A90CA8FFF78E
:106FC000ADFEDDE90C704D460026834620780007B3
:106FD0000AD4AB4500DA5D4601A8012D04DD411954
:106FE00011F8011C302907D04F4502DA17F1040FC0
:106FF00004DA012082460FE06D1EEEE7002F02DC6E
:10700000ED1B3E4403E0781CA84200DD7D1CB81B4C
:1070100000F1010A4FF000472078000703D4AA4589
:1070200001DB4FF0FF3A0021B7F1004F0DF14308AB
:107030008DF8431024D002202B23002F01DA7F4249
:107040002D230A21021EA0F1010000DC5FB197FB95
:10705000F1FC97FBF1F201FB1C7C17460CF1300CA4
:1070600008F801CDEEE7A8F10100037021880905B9
:1070700001D5452100E06521A0F1010800F8011CBF
:1070800009980FA9A1EB0807FF1D00B101204119C4
:1070900001EBEA70A1693844081A401EA06120780B
:1070A000C00602D42046FFF745FC099828B1D4E970
:1070B00001219047206A401C20622078C00622D51A
:1070C0002046FFF737FC1EE0002E04DBB34502DD4F
:1070D00001A8805D00E03020D4E901219047206ABA
:1070E000401C2062761CAAF101005FEA000A0AD166
:1070F00000F072F8C0680168405CD4E90121904753
:10710000206A401C2062281EA5F10105DCDC07E096
:10711000D4E9012118F8010B9047206A401C206235
:10712000381EA7F10107F3DC2046FFF719FC032006
:1071300011B043E601694A1C02610878704700B546
:107140008FB0CDE901310021059105497944CDE9A0
:10715000031011466846FFF751FC0FB000BD000058
:10716000E5FFFFFF0A6802F8010B0A6070470000A4
:10717000074B70B50D467B44FFF7E1FF04462846F8
:1071800000F022F910B14FF0FF3070BD204670BD05
:10719000EBADFFFF4FF000020429C0F0128010F0A9
:1071A000030C00F01781CCF1040CBCF1020F18BFE6
:1071B00000F8012BA8BF20F8022BA1EB0C0100F076
:1071C00009B95FEAC17C24BF00F8012B00F8012B4C
:1071D00048BF00F8012B7047004870472402002088
:1071E00030B5B0F10A024FEA900E71F100034EEA99
:1071F000817EB0EB0E0061EB91014FEA101E4EEA6A
:10720000017E10EB0E0041EB11114FEA102E4EEAF9
:10721000016E10EB0E0041EB11214FEA104E4EEAC9
:10722000014E10EB0E0041EB1141401841F10001FD
:107230004FEAD00040EA41704FEAD10110EB8005DF
:107240004FEA810444EA907444EB01046D1944EB65
:107250000404521BA3414FF0000348BF0A3200D57B
:1072600030BD401C41F1000130BD00002DE9F0416E
:107270001F46044603260168072A01F4006004DB68
:1072800008B116A505E016A503E008B115A500E0B4
:1072900015A521F010002060A069C01EA0610FB1EB
:1072A000401EA0612046FFF745FB4FB1D4E9012104
:1072B00038469047206A401C2062C01C206206E0CD
:1072C000206AFAE7D4E9012115F8010B9047761EF0
:1072D000F8D22046FFF744FBBDE8F0814E414E0056
:1072E0006E616E00494E4600696E66002DE9F047FA
:1072F000814616468AB0334878440DC88DE80D00A3
:1073000030487844801C03AC0DC884E80D0041F679
:107310009B300844372190FBF1F290FBF1F5A5F189
:10732000800501FB12041B3C02D56442012000E0F1
:107330000020DFF890A080460027FA44AAF1BE0A98
:107340000DE0E00709D03246684607EB47010AEB3B
:10735000810100F05CFB8DE8070064107F1C002CAD
:10736000EFD1184F7F44AC3F18E0E80714D007EB8B
:1073700004100DF1180A90E80E008AE80E00C068AB
:10738000F04201D198190890324606A903A800F0EE
:107390003EFB03AB83E807006D10641C002DE4D1B5
:1073A00032466946B8F1000F03A802D000F01BFB7B
:1073B00001E000F02CFBC9E90001C9F808200AB07F
:1073C000BDE8F087802C0000007B00F08000704753
:1073D0004FF0000200B5134694469646203922BF6E
:1073E000A0E80C50A0E80C50B1F12001BFF4F7AFB9
:1073F000090728BFA0E80C5048BF0CC05DF804EB9B
:10740000890028BF40F8042B08BF704748BF20F808
:10741000022B11F0804F18BF00F8012B70470000BD
:1074200000487047040200207546FFF7F9FFAE469A
:1074300005006946534620F00700854618B020B580
:10744000F8F7E2FEBDE820404FF000064FF00007DD
:107450004FF000084FF0000B21F00701AC46ACE8FC
:10746000C009ACE8C009ACE8C009ACE8C0098D4669
:10747000704710B50446AFF300802046BDE81040C9
:10748000F8F7ADBE4FF0013C50F8042B51F8043B27
:107490009A4221D1A2EB0C03934313EACC1317D1E8
:1074A00050F8042B51F8043B9A4215D1A2EB0C037F
:1074B000934313EACC130BD150F8042B51F8043B3F
:1074C0009A4209D1A2EB0C03934313EACC13DBD00D
:1074D0004FF00000704700BFD01A01BAB1FA81F135
:1074E00001F0180122FA01F0CB40C1F12001DBB21A
:1074F000C0B2C01A2CFA01F3D11A914311EAC31198
:10750000E6D170475FEA400C08BF91F0000F4FEAE8
:107510008C234FEAC12243EA51514FEA1C5018BF55
:1075200000F5F0404FEA300018BF41F000415FEA3B
:107530006C5C00F02980BCF1FF3F08BF40F0804048
:107540007047130C06BF12044FF0100C4FF0000CE4
:10755000130E04BF12020CF1080C130F04BF12012A
:107560000CF1040C930F04BF92000CF1020CD30F2A
:1075700004BF52000CF1010C11464FF00002A0F1C3
:107580001F00A0EB0C00704711F0004F08BF7047C0
:1075900031F000413FF4D5AF0B0C06BF09044FF0AA
:1075A000100C4FF0000C0B0E04BF09020CF1080C7C
:1075B0000B0F04BF09010CF1040C8B0F04BF8900F1
:1075C0000CF1020CCB0F04BF49000CF1010CCCF103
:1075D0002003A0EB0C0022FA03F302FA0CF241EABA
:1075E000030100F10100704720F07F4C80EA0300A6
:1075F00023F07F47ACEB070303F57C5300F000401A
:1076000003F1FF032DE980494FEA154B09B44FEA16
:10761000144325EA0B4E24EA03480FF2042606EB36
:10762000132749083E785FEA320203FB0667C7F575
:10763000000707FB06F64FEA54374FEAD64606F135
:10764000020607FB066CCCF1005C4FEA1C472CEAF3
:10765000074C07FB06F40CFB06F504EB15464FEA56
:10766000961634BF00204FF000404FEAD13706FB9A
:1076700007FC4FEA1C4C0CFB0BF7D21B03FB0CF76F
:1076800061EB07010CFB0EF7B0EB074072EB174202
:107690000CFB08F734BFA2EB0742B2EB074261EBE9
:1076A00017414FEA0C444FEA910706FB07FC4FEAEB
:1076B0001C4C0CFB0BF7B0EBC74072EB573203FBD3
:1076C0000CF734BFA2EBC742B2EBC74261EB5731B4
:1076D0000CFB0EF7B0EBC70072EB57720CFB08F710
:1076E00034BFA2EBC702B2EBC70261EB5771039F35
:1076F0004FEA816141EA921104EBCC044FEAD137A1
:107700004FEA826206FB07FC42EA90124FEA806071
:107710004FEA1C4C0CFB0BF7D21B03FB0CF761EB85
:1077200007010CFB0EF7B0EB074072EB17420CFBA6
:1077300008F734BFA2EB0742B2EB074261EB1741F7
:107740004FEA8C554FEA910704EB9C2406FB07FC9B
:107750004FEA1C4C0CFB0BF7B0EBC74072EB5732F7
:1077600003FB0CF734BFA2EBC742B2EBC74261EB9D
:1077700057310CFB0EF7B0EBC70072EB57720CFBE6
:1077800008F734BFA2EBC702B2EBC70261EB577137
:1077900015EB4C254FEA816141EA92114FEA826272
:1077A0004FEAD13742EA901206FB07FC44F100048D
:1077B0004FEA80604FEA1C4C0CFB0BF7D21B03FB1B
:1077C0000CF761EB07010CFB0EF7B0EB074072EB17
:1077D00017420CFB08F734BFA2EB0742B2EB07429B
:1077E00061EB174115EB1C154FEA813141EA9241DB
:1077F0004FEA823242EA90424FEA80304FEA0C76FA
:1078000044F1000448EA03434EEA0B484FF0000EEF
:10781000B2EB080C71EB030724BF624639464EEB0E
:107820000E0E4FF0000B0018524149414BEB0B0B71
:10783000B2EB080C71EB03077BF1000B24BF62462F
:1078400039464EEB0E0E4FF0000B001852414941E5
:107850004BEB0B0BB2EB080C71EB03077BF1000B4E
:1078600024BF624639464EEB0E0E51EA020718BF9E
:1078700046F0010616EB0E7655F1000254F10001B8
:1078800003D5BDE88901BDE80088BDE88901BDE8F0
:107890000048B619524141EB0101A3F101037047C1
:1078A00080807F7E7D7C7B7A79787776767574733D
:1078B000727171706F6E6E6D6C6C6B6A6A696868FC
:1078C000676666656464636362616160605F5F5E92
:1078D0005E5D5D5C5C5B5B5A5A5959585857575608
:1078E000565555555454535352525251515050506D
:1078F0004F4F4F4E4E4D4D4D4C4C4C4B4B4B4A4ABF
:107900004A49494948484847474747464646454502
:10791000454444444443434343424242424141413B
:10792000002B26D4770021D01CB54FEA370703B4CB
:107930004FF010004FF010014FF000000FBCBDE8F9
:1079400010400BF1010BBBF1010F08BF5FEA1707F5
:1079500022BF12F1010211F101014FF0004143F188
:10796000000300F0004043EA00007047F9D35708D5
:10797000DAE746EA064613F1400F4FEA16461FDDE6
:1079800013F1200FDFBF16430A46002120335B426C
:10799000C8D0C3F1200746EA064602FA07F74FEAC5
:1079A000164646EA0706C3F1200722FA03F201FA57
:1079B00007F721FA03F14FF0000342EA0702B1E7AB
:1079C00046EA020646EA06464FEA164646EA010637
:1079D000BCBF46EA0646360C4FF000034FF00002EB
:1079E0004FF000019EE72DE9C048934630B491E87E
:1079F000380007C831EA400C48BF34EA430C03D5CD
:107A0000FFF7F2FDFFF78CFFF0BCBDE800882DE921
:107A1000C048934630B491E8380007C810F0804F52
:107A200008BF13F0804F03D100F005F8FFF778FF8F
:107A3000F0BCBDE8008820F07F4780EA030023F017
:107A40007F4C07EB0C03A3F57C5300F00040A3F13F
:107A5000FE0392F0000F00F0B38095F0000F00F0ED
:107A600077802DE901494FEA11404FEA144621EA97
:107A7000004800FB06FC24EA064708FB06F607FB65
:107A800008F800FB07F718EB06484CEB164C4FEADA
:107A9000124B18EB07484FEA15464CEB174022EA09
:107AA0000B4E0BFB06FC25EA06470EFB06F607FB12
:107AB0000EFE0BFB07F71EEB064E4CEB164C4FF081
:107AC00000061EEB074E4CEB174B18EB0B0840F172
:107AD000000018EB0E0B58EB000840F100008F1A65
:107AE0004FF000013CBFC943661B14BFB5EB040C4B
:107AF00000213CBFC943F61B4FEA17444EEA8E0EE5
:107B000027EA04454FEA1C4704FB07622CEA074CAE
:107B100005FB07F70CFB05F604FB0CFC16EB074610
:107B200042EB174216EB0C4642EB1C421BEB0606DF
:107B300058EB0202414146EA9E0601D5BDE80189A3
:107B4000B619524141EB0101A3F10103BDE80189DE
:107B50004FEA14454FEA114724EA054621EA074C4B
:107B600005FB07F406FB07F70CFB06F105FB0CFC15
:107B700011EB074144EB17444FEA124711EB0C415C
:107B800044EB1C4422EA074C05FB07F206FB07F70F
:107B90000CFB06F605FB0CFC16EB074642EB174206
:107BA00016EB0C4642EB1C456A1854F1000148BF25
:107BB0007047B619524141EB0101A3F1010370472F
:107BC00095F0000F37D04FEA11424FEA144721EAEF
:107BD000024624EA074C02FB07F106FB07F70CFB01
:107BE00006F402FB0CFC14EB074441EB17414FEA8F
:107BF000154714EB0C4441EB1C4125EA074C02FBF2
:107C000007F506FB07F70CFB06F602FB0CFC16EB70
:107C1000074645EB174516EB0C4645EB1C4212197F
:107C200051F1000148BF7047B619524141EB0101C3
:107C3000A3F1010370474FEA14454FEA114724EAC4
:107C4000054621EA074C05FB07F106FB07F70CFB8D
:107C500006F24FF0000605FB0CFC12EB074241EB6D
:107C6000174112EB0C4251EB1C4148BF7047921870
:107C700041EB0101A3F101037047490050EAC12023
:107C800018BF04204A0D18BF40F0010040F2FF72F7
:107C9000B2EB515F08BF40F00200012808BF052089
:107CA00070472DE9F0414F1E00EBC7010446D1E9B2
:107CB000000115461E4637F006020DD02A4633460F
:107CC00000F092FC7F1E04EBC703D3E9002300F011
:107CD0006BFA37F00602F1D1022F25D0042F13D012
:107CE000062F18BFBDE8F0812A46334600F07CFC21
:107CF000D4E90A2300F058FA2A46334600F074FC0F
:107D0000D4E9082300F050FA2A46334600F06CFC10
:107D1000D4E9062300F048FA2A46334600F064FC12
:107D2000D4E9042300F040FA2A46334600F05CFC14
:107D3000D4E9022300F038FA2A46334600F054FC16
:107D4000D4E90023BDE8F04100F02EBA012201F091
:107D50001CBA00F029BA0000024A0020110701F005
:107D600014BA000001FDFFFF30380A2801D20120BB
:107D700070470020704700002DE9F84F04460D467B
:107D800021F0004000917349814211DC7249884220
:107D900001DC06D12CB120462946BDE8F84FFFF79B
:107DA000D5BF6E48002DCCBF6D496E49BDE8F88F38
:107DB0006D49814211DD6D498142D8BF4FF0FF36D8
:107DC0006DDD20462946FFF758FF042808BFFFF75E
:107DD000C3FF20462946BDE8F88F6549654F25F069
:107DE0000045814233DD6449814219DD0026324677
:107DF0004FF080432046294600F0D6F980468A4657
:107E000001222046294601F0C0F900223B4600F03D
:107E1000F5FC4246534600F077FA04460D463EE034
:107E200001260022BA463B462046294600F0BCF90E
:107E300080460F46002253462046294600F0DEFCCD
:107E400042463B4600F060FA04460D4627E04B49A7
:107E500081421BDDDFF828A102260022534620467E
:107E6000294600F0C1FB00223B4600F09DF9804608
:107E70000F46002253462046294600F0BFFC4246EA
:107E80003B4600F041FA04460D4608E00326224630
:107E90002B4600203B4900F037FA04460D462246A7
:107EA0002B461046194600F09FFB8B468246024641
:107EB0000B4600F099FB07460246334888460B46BE
:107EC00006217844FFF7EDFE52465B4600F08CFB3E
:107ED00082462E488B463A46434605217844FFF7B2
:107EE000E0FE3A46434600F07FFB02460B46002E7A
:107EF000504659460CDA00F057F922462B4600F05E
:107F000073FB01B022462B46BDE8F04F00F06ABC7F
:107F100000F04AF922462B4600F066FB1C4A7A44E0
:107F200002EBC603D3E9002300F068FC22462B468F
:107F300000F064FC174A7A4402EBC603D3E900233D
:107F400000F050FC009A002AB8BF81F00041BDE863
:107F5000F88F0000000010440000F07F182D4454FA
:107F6000FB21F93FFB21F9BF0000DC3F0000203E70
:107F70000000F33F0000F03F0000E63F00800340B8
:107F80000000F83F0000F0BF02200000C01F00000A
:107F90005E1F0000261F00002DE9F04D9446CCF135
:107FA000000423F000464CEA0404524F46EAD4741D
:107FB0009A46884621F00042BC4206D8454240EA33
:107FC000050442EAD474BC4204D9BDE8F04D6246CF
:107FD000FFF7BFBEAAF14055A5F17F6555EA0C0435
:107FE0000BD0022404EAAA74434DDFF810E144EAFE
:107FF000D87452EA000B04D00CE0BDE8F04DFFF756
:10800000BBBE002C14BF012CBDE8F08D022C30D07B
:10801000032C32D056EA0C0B0AD0BE4220D1BA4211
:1080200009D126F0804622F080423346114617E0FF
:1080300000291ADB25E0DFF8C8B0FB44002C04BFA0
:10804000DBE90001BDE8F08D012C02BFDBE9000196
:1080500081F00041BDE8F08D022C0AD0032C0CD039
:10806000BA4212D1B8F1000F0BDA23482549BDE816
:10807000F08D28462449BDE8F08D28467146BDE8BC
:10808000F08D1D482149BDE8F08D921B12153C2A48
:10809000C4BF19481D490EDCBAF1000FBEBF12F172
:1080A0003C0F0020014606DB624600F02DF921F06E
:1080B0000041FFF761FE002C08BFBDE8F08D012CE8
:1080C00004BF81F00041BDE8F08D114A114B022C34
:1080D00007D000F093FB2A46BDE8F04D0A4B00F0B4
:1080E0008DBB00F08BFB2A46BDE8F04D064B00F03F
:1080F00079BB00000000F07F182D4454FB2109C01B
:10810000BA1E0000FB21F9BFFB210940FB21F93F0A
:10811000075C143326A6A13C10B500290AD00878C4
:10812000002807D005487844FFF7ACF9002801D0B3
:10813000002010BD0248784410BD0000DE1E000083
:10814000D61E000021F00042A2F16052B2F5801F5D
:1081500001F0004328BFD2F17F6C0BD95FEA001C0D
:1081600043EAC20242EB507018BF704728BF20F0AC
:1081700001007047B2F5801FBCBF184670474FEA38
:10818000410C1CF5001F02D2084600F014BF70B568
:1081900000F0D4FA00000089FFF7F6BF4FF000406E
:1081A000A0F580007047000010B591EA030F48BFAA
:1081B00083F0004300F12A83841A71EB030C05D28B
:1081C000121943EB0C03001B61EB0C01DFF824E1F7
:1081D0004FEA1154A4EB135C1EEA430F18BF9EEA4A
:1081E000445F73D023EA0E03DCF1200E21EA045130
:1081F00043F4801332D322FA0CFE10EB0E0023FA64
:108200000CFE41EB0E01CCF1200E03FA0EFE10EB3A
:108210000E0051F10001B1F5801FCCF1200E32D2D9
:1082200001EB045112FA0EF2BDE8104058BF70473E
:10823000401C38BF5FEA420218BF7047002814BFD5
:1082400020F0010041F100014FEA410313F5001F46
:1082500038BF7047A1F1C04100F0BEBA012A43EB1C
:108260000302ACF1200CDCF11F0E32BF4FF0000E08
:1082700023FA0CF310EB030041EB0451B4EB115F54
:10828000D0D0A1EB045101F5801149085FEA30001C
:1082900001EB04510ED350F1000038BF12FA0EFE6C
:1082A00008D1BDE81040C9E7401C38BF5FEA420270
:1082B000CAD1C3E7BDE810404FEA410313F5001FE0
:1082C00038BF7047A1F1C04100F086BA9EEA445F12
:1082D00008D011EA5E0FBDE8104004BF01F0004174
:1082E00000207047BDE8104070B500F027FA00BFCD
:1082F00064FBBE3E0000E0FF02494FF0000000F0CA
:1083000012BF00BF0000F87F2DE9C04130B4DFF894
:10831000A0C23CEA111418BF3CEA131400F0EC8030
:1083200081EA03051CEA111444EAD57418BF1CEA5B
:10833000131500F0C780A4EB05044FF0004545EA93
:10834000C12145EAC32341EA505143EA525304F1A3
:108350007F74994204F500344FEAC0204FEAC222EC
:1083600008BF904200F09C804FEA13650FF2401660
:10837000765D4FEA134506FB05F7C7F1807706FBEC
:1083800007F74FEAD737A7FB03687642C8F580386E
:10839000A7FB06CE38BFA8F1010807FB08E64FF09F
:1083A000000EA6FB028CE6FB03CEDCF1000CCEF146
:1083B000004E38BFAEF1010EA6FB0C584FF000077F
:1083C0004FF00005E6FB0E87A1FB08C6A0FB07CE19
:1083D00016EB0E0645F10005E1FB076515F1E04ED1
:1083E0007EBFA4F580345FEA46066D4116F1800732
:1083F00045F100054FEA17274FEA066647EA056789
:10840000A6F1DE46B6F1805F4FEA15251FD9384642
:1084100024F0010C05EBC471BCF1FE6F01EB0C11F3
:1084200002D8F0BCBDE8008124425CBF01F5801E8B
:108430009EEAC47F02D4F0BCBDE80081244238D457
:10844000F0BCA1F1C041BDE8004100F0C5B94FEA60
:10845000D22242EA43524FEAD323A7FB02864FEAD5
:10846000D02040EA415007FB03661EEA0E0F4FEA98
:10847000D12105FB026658BFA6EB0056B6EB0056AD
:108480004FEA520E4EEAC37E18EB0E0E56EB530E19
:10849000BDD518EB02085E417F1C55F10005B6E71B
:1084A0004FF480154FF000074FF000064FF0000822
:1084B000ADE7F0BC4FF0000001F1C04101F0004118
:1084C000BDE8008111EA0C1F0CEA131500D00CE086
:1084D00013EA0C1F00F025804FF00000F0BC81EA89
:1084E000030101F00041BDE80081F0BCBDE800419E
:1084F00081EA030100F070B9F0BCBDE8004170B53D
:1085000000F01CF9097EFC3E00F007B881EA030187
:108510004FF0000001F00041704781EA030100F0D4
:108520005BB9F0BCBDE800414FF000002149704745
:10853000FFFDFBF9F7F5F4F2F0EEEDEBE9E8E6E428
:10854000E3E1E0DEDDDBDAD8D7D5D4D3D1D0CFCDAF
:10855000CCCBCAC8C7C6C5C4C2C1C0BFBEBDBCBBE8
:10856000BAB9B8B7B6B5B4B3B2B1B0AFAEADACABE3
:10857000AAA9A8A8A7A6A5A4A3A3A2A1A09F9F9EBD
:108580009D9C9C9B9A99999897979695959493936F
:10859000929191908F8F8E8E8D8C8C8B8B8A898906
:1085A0008888878786858584848383828281818089
:1085B0000000FF070000F87F10F0004248BF404273
:1085C000B0FA80F310FA03F10AD0C3F11D0303F5EA
:1085D00080634FEA415002EB035202EBD121704716
:1085E0004FF0000070470000DFF848C170B51CEA8A
:1085F000111E1EBF1CEA13159EEA0C0F95EA0C0F04
:1086000000F06F8081EA030423EA4C134EEAD47E23
:1086100021EA4C1141F4801143F48013AE44A1FBD4
:10862000024CA0FB0365AEF17F7E361955EB0C05BD
:10863000A1FB034C4CF10003A0FB021C16EB0C0643
:10864000654153F10003094218BF46F0010613F4D7
:10865000007F0BD14FEA03314FEA0530340341EA82
:10866000155140EA16506FF003020AE04FEAC321A9
:108670004FEAC520F40241EA555140EA56506FF0E6
:10868000020202EB2E4201EB025585EACE710AD0BE
:108690005FEA440C18BF24F0004450F1000041F19F
:1086A000000120EAD47040F2FE7C624500D270BD29
:1086B000A84214BF4FF080444FF04044002E08BF42
:1086C0000024BEF1806FA8BFA1F1C041BDE8704099
:1086D00080F282804FF0000001F1C04101F00041C2
:1086E00070479EEA0C0F0CEA131518BF95EA0C0FA1
:1086F00006D04FF0000081EA030E0EF0004170BD7D
:1087000000F01CF88900013E00F007B800F009B83D
:108710004FEA430C5FEA5C5C08D081EA030100F099
:108720005BB84FEA410C5FEA5C5CF6D14FF00000A9
:10873000014970470000FF070000F87F0EF1020EAC
:108740002EF0030E5EF8046B364205D4012A43EB8B
:10875000030515F5001F12D8012841EB010C1CF58B
:10876000001F0CD80ED14FEAD17C15F5001F0CEB81
:108770004C0C0CF1020C08BF4CEBD37C04E04FF026
:10878000080C01E04FEAD37C0CEB4C0526FA05F609
:1087900006F00706B6F1040C06D20EEB860CBDE817
:1087A00070404CF0010C6047DFE80CF0090B02024E
:1087B0004FF000414FF00000A1F5002170BD1946B7
:1087C0001046012851EB010418BFD4F5001484BFF2
:1087D000002001F0004170BD0808A0F500114FEA2B
:1087E0003101704791EA030F10B581F000413FF568
:1087F000E3AC83F0004300F009B8000010B591EA43
:10880000030F48BF83F000433FF5D6AC841A71EBE9
:10881000030C07D212198CF0004C43EB0C03001B25
:1088200061EB0C01DFF8A4E14FEA1154A4EB135CF7
:108830001EEA430F18BF9EEA445F00F0B08023EAAF
:108840006E03524221EA0451C3EB6E0338BF5B1E34
:10885000DCF1200E25D322FA0CFE10EB0E0043FAB9
:108860000CFE41EB0E01CCF1200E03FA0EFE10EBD4
:108870000E0051F10001CCF1200E29D412FA0EF2B3
:1088800001EB0451BDE8104058BF7047401C1CBFAD
:10889000B2F1004F704700280CBF491C20F00100C6
:1088A000704712EB020E43EB030218BF4FF0010EAC
:1088B0004EEA4202ACF1200CDCF11E0E54D943FA10
:1088C0000CFE10EB0E0051F1FF31CCF11E0ED5D590
:1088D0000EF1010E12FA0EFE404141EB010101EBD7
:1088E000445C5FEA5C5C10D910EBDE7001EB045174
:1088F00038BFBEF1004FBDE8104018BF70470028D8
:108900000CBF491C20F00100704730D24FEAD42C34
:1089100011F5001124F400641BD0B1FA81F20B3A76
:10892000A41AA41ED2F12003914030FA03F3194394
:10893000904001EBCC71002C01EB0451BDE81040DC
:10894000A8BF704701F1C0414FF0000001F00041A5
:108950007047B0FA80F310FA03F100D110BDE41AA9
:10896000173C4805C90AE4E701EB045110BD491062
:1089700001EB0451BDE810404FEA300002E04FF037
:10898000000170474A0008BF0042F8D0B2F5001F4E
:1089900028BF704701F000414FF0000070479EEA89
:1089A000445F07D011EA5E0FBDE8104004BF00210C
:1089B00000207047BDE8104070B5FFF7BFFE00BF54
:1089C00040DFF63E83F00041104670470000E0FFB4
:1089D00043004FEAD30C4FEA3C0C43401FBF400713
:1089E0000CF1605113F0FE4F70471CF0006F03D183
:1089F00000200CF0004170470CF0004343EA507037
:108A000010B540EACC0000F090FA00BF00000092E0
:108A10004FEA0001FFF7E0BE4FF000414FF00000C9
:108A2000A1F500217047000090EA010F48BF81F0D6
:108A3000004100F10883421A3CBF801A89184FEAAE
:108A4000D0524FF07F4C1CEA410FA2EBD15318BF1C
:108A50009CEA026F00F03B804FF0004C4CEA002093
:108A60004CEA012121FA03FC10EB0C0C1ED202F19E
:108A7000FF325FEA1C2040EBC25038BF70471CF049
:108A80007F0F4FEA400C18BFBCF17F4F38BF7047D3
:108A9000C3F12003994008BF20F00100BCF17F4FD3
:108AA00038BF7047A0F1C04000F085BA4FEA3C00E3
:108AB000000A40EBC25028BF1CF0FF0F4FEA400CE9
:108AC000E6D018BFBCF17F4F38BF7047EAE79CEA99
:108AD000026F05D010EA5C0F08BF00F0004070473D
:108AE00010B500F022FA00BF64FBBE3E401058BF34
:108AF000C0F14040491058BFC1F140418142EFF3FD
:108B0000008070474FF47F0C1CEAD0121EBF1CEA95
:108B1000D11392EA0C0F93EA0C0F00F0858090EAD3
:108B2000010F48BF42F4807240F4000C41F4000091
:108B30002CF07F4120F07F4000B58142A2EB030280
:108B40000FF2081CACEB504EC0F100009EF800E0A4
:108B50004FEA4E0E00FB0EFC38BF49004FEA2C1CBA
:108B600002F5FA020CFB0EF34FEACE1E4FEA112C6F
:108B70004FEAC1210EEB635E42EB22420EFB0CFC7E
:108B80004FEA1C5300FB03114FEA112C4FEA01314D
:108B90000EFB0CFC4FEADC4C00FB0C11C14228BF61
:108BA00009184CEB03335DF804EB10EB410143EB88
:108BB000C250B2F57C0F38BF704729D512F0F00FC4
:108BC0001CBF00F1C04000F000407047008182836C
:108BD0008485868788898B8C8D8E8F9192939596CC
:108BE00097999A9C9D9FA0A2A3A5A7A8AAACAEB056
:108BF000B2B3B5B7B9BCBEC0C2C5C7C9CCCED1D45B
:108C0000D7D9DCDFE2E6E9ECF0F3F7FAFE0000008A
:108C10004FEA400C0CF1807CBCF17E4F28BF7047BE
:108C2000B0F1C04000F0C7B990EA010F0CEAD113CF
:108C300048BF42F48072624538BF634507D213F4DF
:108C40007F0F16D080EA010000F00040704710B599
:108C500000F06BF9097EFC3E00F005B880EA0100E7
:108C600000F00040704780EA010000F0004000F092
:108C7000A2B912F47F0F04BF0248704780EA0100D6
:108C800000F099B90000C07F50EA010C00F1138098
:108C90001CF5000F58BFBCF5000F01D48842704787
:108CA00007D710F5000F58BF11F5000F15D48842F3
:108CB0007047894270471CF5000F04D5BCF5000FC2
:108CC000F7D5814270474FF0807C1CEB400F38BFD6
:108CD0001CEB410F01D28142704710B500F025F91D
:108CE000922449004FF000504FF08051FFF7FEBE34
:108CF00041000B0ED3F19E0208D950F400034FEA55
:108D0000032323FA02F048BF4042704710B500F039
:108D10000CF900BF49922480002070476FF0004298
:108D200082EA200070470000C10DD1F19E0206DBEF
:108D30004FEA002343F0004323FA02F07047004259
:108D400007D54FEA4001B1F1FE4F02D24FF00000CB
:108D5000704710B500F0E9F8499224800020704770
:108D60006FEA20007047000010F0004148BF404209
:108D7000B0FA80F310FA03F2C3F19D030BD051EA6D
:108D8000C35101EB1220530638BF704700F10100B8
:108D900008BF20F001007047B0FA80F310FA03F228
:108DA000C3F19D030AD0D90501EB1220530638BF49
:108DB000704700F1010008BF20F00100704700007B
:108DC00050EA010C00F113801CF5000F58BFBCF5F0
:108DD000000F01D48842704707D710F5000F58BF25
:108DE00011F5000F15D488427047894270471CF571
:108DF000000F04D5BCF5000FF7D5814270474FF046
:108E0000807C1CEB400F38BF1CEB410F01D281422C
:108E1000704710B500F089F8922449004FF00050D7
:108E20004FF08051FFF762BE4FF47F0C1CEAD01266
:108E30001EBF1CEAD11392EA0C0F93EA0C0F00F04C
:108E4000478090EA010F48BF42F480724FF0004C17
:108E50004CEA00204CEA012102EB0302A0FB0113C3
:108E6000A2F50002002918BF43F001035B0028BFF0
:108E70004FEA330342EB22425FEA132C4CEBC25021
:108E80002EBFBCEB436FB2F57C0F70474FEA036C0B
:108E9000BCF1004F08BF20F00100B2F57C0F38BFD5
:108EA00070470BD582F0FF0212F5803FC8BF7047B4
:108EB00000F1C040D8BF00F00040704700F5000C42
:108EC0005FEA4C0C48BF7047B0F1C04000F073B887
:108ED00090EA010F0CEAD11348BF42F48072624558
:108EE00038BF634504D280EA010000F000407047BB
:108EF00010B500F01AF800BF8900013E00F007B875
:108F000000F009B85FEA410C5FEA1C6C08D080EA07
:108F1000010000F050B85FEA400C5FEA1C6CF6D12B
:108F20004FF00040A0F5800070470EF1020E2EF0C9
:108F3000030E5EF8044B244204D44FEA4102B2F11E
:108F40007F4F11D84FEA4003B3F17F4F0CD80ED1B9
:108F50004FEAD07CB2F17F4F0CEB4C0C0CF1020CC1
:108F600008BF4CEBD17C04E04FF0080C01E04FEA65
:108F7000D17C0CEB4C0324FA03F404F00704B4F1A5
:108F8000040C06D20EEB840CBDE810404CF0010C32
:108F90006047DFE80CF0070802024FF00040A0F540
:108FA000800010BD0846420018BFD2F1807288BF11
:108FB00000F0004010BDFF2141EAD050C0057047CD
:108FC00051EA000C00F113801CF5000F58BFBCF5EE
:108FD000000F01D48142704707D711F5000F58BF29
:108FE00010F5000F15D481427047894270471CF577
:108FF000000F04D5BCF5000FF7D5884270474FF03D
:10900000807C1CEB410F38BF1CEB400F01D2884223
:10901000704780EA010081EA000180EA0100FFF761
:10902000F8BE80F0004090EA010F7FF504AD81F0BA
:10903000004100F008B8000090EA010F48BF81F03D
:1090400000413FF5F8AC421A04D882F00042A0EB90
:10905000020011444FEAD0524FF07F4C1CEA410FFE
:10906000A2EBD15318BF9CEA026F4AD04FF0004CDC
:109070004CEA00204CEA012121FA03FCB0EB0C0C75
:109080000FD412F0FE0F36D05FEA4C001DD500124F
:1090900040EBC25038BF70471CF03F0F18BF7047FD
:1090A0000BE0A2F101025FEA1C2040EBC25038BF86
:1090B00070471CF07F0F18BF7047C3F12003994021
:1090C00014BF401E20F00100704780084FEA1223B1
:1090D00008BF7047B0FA80FCA2EB0C02CCF1280C60
:1090E00060FA0CF093EA122F04BF00EBC2507047F5
:1090F0004FEAC3707047130A5FEADC1008BF70477D
:10910000F6E79CEA026F04D010EA5C0F08BF00206B
:10911000704710B5FFF709FF40DFF63E81F00040D1
:109120007047FDF7D1BE0CF00F03092B08BF0820D4
:1091300000F059800A2B0BD0082B18BF704708BFCE
:109140001CF0400F0AD04FF000004FF000017047B4
:109150001CF0400F18BF4FF0004070471CF0100F7C
:1091600008D020F0704300F07F4242EAD3014FEA7A
:109170004370704700F0604021F07F4242EA0002F5
:1091800001F07F4040EA727070474FF0FF0C4CF4E2
:10919000E06C1CEA11531CBF9CEA030C9445C2BF4F
:1091A000DA4201EB02517047002B0DD0BCF1000FE9
:1091B0000FD0002A01F00041A4BF41F0E04141F08E
:1091C0007F614FF00000704701F000414FF0000058
:1091D000704750EA01334FF09B0C18BF4CF0806C85
:1091E0007FF48AA870471CF4801F11D01CF4E02F74
:1091F00003D06FEACC31490070474FF04050EFF395
:10920000008222F0704242EA000282F30088704736
:109210004FF0000070470000680000047600540121
:10922000F7FD000175191A0C6A231B1C1F207274AC
:10923000433B4138393A6B6C376F06246D6E7000D2
:109240008300000000080000000100183200050043
:10925000000020410000D242295C0F3E9A99993EBD
:109260003333733F295C0F3E000070000000002480
:10927000000000020003000000650054FFEF000042
:10928000FA80000B12820001030C30C30E8C8CE9B3
:1092900014D5400213710F8E3883F8833000F883A1
:1092A000258EF8833000F883FFFFFFFF0FFEA9D65D
:1092B000240004001A8279A10000003CFFFF000096
:1092C0000010000038836FA2003E03304000000011
:1092D00002CAE3093E8000002000000000000000F8
:1092E0004000000060000000000C0000000C186E40
:1092F000000006920A16C0DFFFFF0256FD8CD377EE
:10930000FFE1C496E0C5BEAA00000000FFFF0B2BE2
:1093100000001657000003594000000000001DFA2D
:1093200000026C1D000000003FFFDFEB003EB3B603
:10933000000D227800002F3C00000000001942B50B
:10934000000039A20000B365D90E9FC91DCF4C346F
:1093500030000000500000003BB67AE800640000D6
:1093600000C8000000000000100000001000FA9289
:109370001000225E000D229F00010000003200005C
:10938000FF46000063D400001000000004D6000077
:1093900004CC000004CC000000001072000000406B
:1093A00000000000000000000006000200050007A9
:1093B0000000000000640000000000000000000544
:1093C0000005006400200000000000000000000014
:1093D000000040000000030000000032F898000088
:1093E000FF650000830F0000FF9BFC0000000000F1
:1093F000000000000000000000000000000000006D
:10940000000000000000000000000000000000005C
:1094100000000000000010004000000000000006F6
:109420000000B26A000200000001FB830068000037
:1094300000D9FC007CF1FF83000000000065000003
:10944000006403E80064002800000025000000001C
:1094500016A000000000100000001000002F000007
:10946000000001F40000100000280000FFFF45810B
:10947000FFFFFA7200000000000000000044000539
:109480000005BAC6004778A20000000100000000F5
:1094900000000600000000140000254D002F706D34
:1094A000000005AE000C02D000000000000000002B
:1094B0000000000000000000001B00000000000091
:1094C0000000000000000000006400000008000030
:1094D000000000000000000000000000000000008C
:1094E000000000000000000000000000000000007C
:1094F000000000000000000000000000000000006C
:10950000000000000000000000000000000000005B
:10951000000000000000000000000000000000004B
:109520000000000000000000001B00000000000020
:1095300000000000000E000E00000AC7000400003A
:1095400000000032FFFFFF9C00000B2B0000000218
:109550000000000100000064FFE5000000000000C2
:1095600000000000000000000000000100000000FA
:1095700000010000000000000001800000018000E8
:1095800000018000002426D300000000000000003D
:10959000000600100096003C0000000000000000E3
:1095A00000000000000000000C0A4E68CDCF7709D3
:1095B00050166759C619CE82000000000000000056
:1095C000000000000000000000000000000000009B
:1095D00017D7840003000000000000000000000016
:1095E000C7938F9D1E1B1C19000000000000000087
:1095F000000000000000000000000000000000006B
:109600000203188500004000000000030000000372
:10961000000000000000000040000000000000000A
:10962000000000000000000000000000000000003A
:10963000000000000000000000000000000000002A
:10964000000000000000000000000000677DDF7ED9
:1096500072902E554CF6E6880000000000000000D5
:109660000000000000000000D8DCB4B8B0D8B9ABEE
:10967000F3F8FAB3B7BB8E9EAEF132F51BF1B4B876
:10968000B08097F1A9DFDFDFAADFDFDFF2AAC5CD67
:10969000C7A90CC92C97F1A989264666B28999A950
:1096A0002D557DB0B08AA896365676F1BAA3B4B2DD
:1096B00080C0B8A89711B28398BAA3F024084410C8
:1096C0006418B2B9B49883F1A329557DBAB5B1A392
:1096D0008393F0002850F5B2B6AA839328547CF106
:1096E000B9A3829361BAA2DADEDFDB819AB9AEF563
:1096F000606870F1DABAA2DFD9BAA2FAB9A382928D
:10970000DB31BAA2D9BAA2F8DF85A4D0C1BBAD8340
:10971000C2C5C7B8A2DFDFDFBAA0DFDFDFD8D8F16C
:10972000B8AAB38DB4980D355DB2B6BAAF8C9619A0
:109730008F9FA70E161EB49AB8AA872C547CBAA481
:10974000B08AB691325676B28494A4C808CDD8B8FF
:10975000B4B0F19982A82D557D98A80E161EA22CA2
:10976000547C92A4F02C5078F184A898C4CDFCD8F5
:109770000DDBA8FC2DF3D9BAA6F8DABAA6DED8BA62
:10978000B2B68696A6D0F3C841DAA6C8F8D8B0B467
:10979000B882A892F52C548898F135D9F418D8F1EC
:1097A000A2D0F8F9A884D9C7DFF8F883C5DADF6951
:1097B000DF83C1D8F40114F1A8824EA884F311D13B
:1097C00082F5D992289788F109F41C1CD884A8F353
:1097D000C0F9D1D99782F129F40DD8F3F9F9D1D98B
:1097E00082F4C203D8DEDF1AD8F1A2FAF9A884986D
:1097F000D9C7DFF8F8F883C7DADF69DFF883C3D8A1
:10980000F40114F198A8822EA884F311D182F5D91D
:1098100092509788F109F41CD884A8F3C0F8F9D1C4
:10982000D99782F149F40DD8F3F9F9D1D982F4C46A
:1098300003D8DEDFD8F1AD8898CCA809F9D9829297
:10984000A8F57CF1883ACF944A6E98DB6931DAAD9D
:10985000F2DEF9D88795A8F221D1DAA5F9F417D963
:10986000F1AE8ED0C0C3AE82C684C3A88595C8A50C
:1098700088F2C0F1F4010EF18E9EA8C63E56F55452
:10988000F18872F40115F19845856EF58E9E048875
:10989000F142985A8E9E068869F4011CF1981E11B7
:1098A00008D0F504F11E970202983625DBF9D98518
:1098B000A5F3C1DA85A5F3DFD88595A8F309DAA564
:1098C000FAD88292A8F578F1881A849F2688982180
:1098D000DAF41DF3D8879F39D1AFD9DFDFFBF9F474
:1098E0000CF3D8FAD0F8DAF9F9D0DFD9F9D8F40BBB
:1098F000D8F3879F39D1AFD9DFDFF41DF3D8FAFC55
:10990000A869F9F9AFD0DADEFAD9F88F9FA8F1CCBF
:10991000F398DB45D9AFDFD0F8D8F18F9FA8CAF311
:109920008809DAAF8FCBF8D8F2AD978D0CD9A5DFC7
:10993000F9BAA6F3FAF412F2D8950DD1D9BAA6F372
:10994000FADAA5F2C1BAA6F3DFD8F1BAB2B68696B2
:10995000A6D0CAF349DAA6CBF8D8B0B4B8D8AD844B
:10996000F2C0DFF18FCBC3A8B2B68696C8C1CBC315
:10997000F3B0B48898A821DB718D9D71859521D9AC
:10998000ADF2FAD88597A828D9F408D8F28D29DA4B
:10999000F405D9F285A4C2F2D8A88D9401D1D9F4E6
:1099A00011F2D88721D8F40AD8F28498A8C801D136
:1099B000D9F411D8F3A4C8BBAFD0F2DEF8F8F8F8A8
:1099C000F8F8F8F8D8F1B8F6B5B9B08A95A3DE3C46
:1099D000A3D9F8D85CA3D9F8D87CA3D9F8D8F8F9DA
:1099E000D1A5D9DFDAFAD8B18530F7D9DED8F83089
:1099F000ADDADED8F2B48C99A32D557DA083DFDFDC
:109A0000DFB591A0F629D9FBD8A0FC29D9FAD8A0B6
:109A1000D051D9F8D8FC51D9F9D879D9FBD8A0D0F0
:109A2000FC79D9FAD8A1F9F9F9F9F9A0DADFDFDF81
:109A3000D8A1F8F8F8F8F8ACDEF8ADDE8393AC2CDA
:109A4000547CF1A8DFDFDFF69D2CDAA0DFD9FADB4A
:109A50002DF8D8A850DAA0D0DED9D0F8F8F8DB5528
:109A6000F8D8A878DAA0D0DFD9D0FAF8F8F8F8DB7F
:109A70007DF8D89CA88CF530DB38D9D0DEDFA0D0BB
:109A8000DEDFD8A848DB58D9DFD0DEA0DFD0DED8B3
:109A9000A868DB70D9DFDFA0DFDFD8F1A888902CC1
:109AA000547C98A8D05C38D1DAF2AE8CDFF9D8B00B
:109AB00087A8C1C1B188A8C6F9F9DA36D8A8F9DAF9
:109AC00036D8A8F9DA36D8A8F9DA36D8A8F9DA36C5
:109AD000D8F78D9DADF818DAF2AEDFD8F7ADFA30D1
:109AE000D9A4DEF9D8F2AEDEFAF983A7D9C3C5C787
:109AF000F1889BA77AADF7DEDFA4F8849408A797D6
:109B0000F300AEF29819A488C6A39488F632DFF267
:109B10008393DB09D9F2AADFD8D8AEF8F9D1DAF30A
:109B2000A4DEA7F1889B7AD8F38494AE19F9DAAA57
:109B3000F1DFD8A881C0C3C5C7A39283F628ADDEE4
:109B4000D9F8D8A350ADD9F8D8A378ADD9F8D8F8BA
:109B5000F9D1A1DADEC3C5C7D8A18194F818F2B053
:109B600089ACC3C5C7F1D8B8B4B09786A8319B06F5
:109B70009907AB9728889BF00C201440B0B4B8F03C
:109B8000A88A9A285078B79BA829517924705944FB
:109B90006938644831F1BBAB88002C547CF0B38B3E
:109BA000B8A804285078F1B088B49726A85998BB73
:109BB000ABB38B02264666B0B8F08A9CA8295179CF
:109BC0008B2951798A2470598B2058718A446938BD
:109BD0008B3940688A6448318B30496088F1AC0029
:109BE0002C547CF08CA804285078F1889726A8592A
:109BF00098AC8C02264666F0899CA829517924707D
:109C000059446938644831A98809205970AB113822
:109C10004069A8193148608CA83C415C207C00F167
:109C200087981986A86E767EA999882D557DD8B11A
:109C3000B5B9A3DFDFDFAED0DFAAD0DEF2ABF8F933
:109C4000D9B087C4AAF1DFDFBBAFDFDFB9D8B1F18C
:109C5000A3978E60DFB084F2C8F8F9D9DED8938577
:109C6000F14AB183A308B5839A0810B79F10D8F1C1
:109C7000B0BAAEB08AC2B2B68E9EF1FBD9F41DD88E
:109C8000F9D90CF1D8F8F8AD61D9AEFBD8F40CF1E4
:109C9000D8F8F8AD19D9AEFBDFD8F416F1D8F8AD85
:109CA0008D61D9F4F4ACF59C9C8DDF2BBAB6AEFA7D
:109CB000F8F40BD8F1AED0F8AD51DAAEFAF8F1D82D
:109CC000B9B1B6A3839C08B9B1839AB5AAC0FD30D7
:109CD00083B79F10B58B93F20202D1ABDADED8F1D5
:109CE000B080BAABC0C3B284C1C3D8B1B9F38BA33F
:109CF00091B609B4D9ABDEB0879CB9A3DDF1B38BC3
:109D00008B8B8B8BB087A3A3A3A3B28BB69BF2A341
:109D1000A3A3A3A3A3A3A3A3A3F1B087B59AA3F37B
:109D20009BA3A3DCBAACDFB9A3A3A3A3A3A3A3A360
:109D3000A3A3A3A3A3A3A3A3D8D8D8BBB3B7F1AAC3
:109D4000F9DAFFD9809AAA28B48098A720B7978714
:109D5000A86688F07951F1902C870CA781976293BF
:109D6000F071716085940129517990A5F1284C6CAE
:109D7000870C95188578A38390284C6C886CD8F351
:109D8000A28200F210A8921980A2F2D926D8F188F6
:109D9000A84DD948D896A83980D93CD89580A839FB
:109DA000A68698D92CDA87A72CD8A8899519A980D6
:109DB000D938D8A88939A980DA3CD8A82EA83990F2
:109DC000D90CD8A8953198D90CD8A809D9FFD801B1
:109DD000DAFFD89539A9DA26FFD890A80D8999A875
:109DE00010809821DA2ED88999A83180DA2ED8A847
:109DF00086963180DA2ED8A8873180DA2ED8A882CC
:109E000092F34180F1D92ED8A882F31980F1D92E8E
:109E1000D882ACF3C0A28022F1A62EA72EA9229848
:109E2000A829DAACDEFFD8A2F22AF1A92E8292A8E4
:109E3000F23180A696F1D900AC8C9C0C30ACDED00F
:109E4000DEFFD88C9CACD010ACDE8092A2F24C82AB
:109E5000A8F1CAF235F19688A6D900D8F1FF000022
:109E60004FBB610567ACDD3F182D4454FB21E93F32
:109E70009BF681D20B73EF3F182D4454FB21F93F21
:109E8000E2652F227F2B7A3C075C143326A6813CA7
:109E9000BDCBF07A8807703C075C143326A6913C52
:109EA000C4EB98999999C9BF711623FEC671BCBFBE
:109EB0006D9A74AFF2B0B3BF9AFDDE522DDEADBF26
:109EC0002F6C6A2C44B4A2BF0D5555555555D53F3E
:109ED000FF8300922449C23F6E204CC5CD45B73F59
:109EE000513DD0A0660DB13FEB0D76244B7BA93FD1
:109EF00011DA22E33AAD903F0000000000000000BC
:109F000002400000000000A000000000054000002A
:109F1000000000C8000000000C4000000000409C51
:109F200000000000194000000020BCBE000000003E
:109F300034400000BFC91B8E00000004B540000083
:109F4000504BCFD06607E2CF010000006C4100000B
:109F50003E8251AADFEEA73401000000D942000082
:109F6000DCB5A0E23A301F97FFFFFFFFB4450000C9
:109F7000FD25A0C8E9A3C14FFFFFFFFFFF3F000081
:109F80000000008000000000FF3F00000000008093
:109F90000000000050726F647563742049442072A1
:109FA000656164206173203020696E646963617447
:109FB00065732064657669636520697320656974DB
:109FC00068657220696E636F6D70617469626C653B
:109FD000206F7220616E204D5055333035302E0D7C
:109FE0000A00000020A0000800000020200100005E
:109FF0006C01000840A10008200100204807000073
:10A00000880100081C00000043000000F8FFFFFF6B
:10A010000C0000000E0000000F0000002E000000E9
:10A0200000A24A0400000000000000000102030436
:10A0300006070809000000000102030401020304EE
:10A0400006070809020406080000000000000000DE
:10A050000000000000000000000000000000000000
:10A060009A99193FCDCCCC3D0000000000000000C3
:10A0700000000000000000000000000000000000E0
:10A0800000000000000000000000000000000000D0
:10A09000000000004600000000000000000000007A
:10A0A00000000000000000000000000000000000B0
:10A0B00000000000000000000000000000000000A0
:10A0C0000000000000000000000000000000000090
:10A0D00000000000000000000000803F00000000C1
:10A0E0000000000000000000FF000000FF00000072
:10A0F00001000000000000002492000818920008EF
:10A10000000000000000000000000000000000004F
:10A11000000000000000000000000000000000003F
:10A120004092000800000000000000000100000054
:10A13000000000000000000000000000000000001F
:0400000508000131BD
:00000001FF
